:040000006F00F00B92
:100004000000000000000000EE050000F005000004
:1000140000000000BC080000000000000000000018
:10002400BC080000BC080000000000000000000044
:100034002216000000000000000200000000000082
:10004400BC080000BC080000BC080000BC0800009C
:10005400BC080000BC080000BC080000BC0800008C
:10006400BC080000BC080000BC080000BC0800007C
:10007400BC080000BC080000BC080000BC0800006C
:10008400BC080000BC080000BC080000BC0800005C
:10009400BC080000BC080000BC080000BC0800004C
:1000A400BC080000BC080000BC080000BC0800003C
:1000B400BC080000BC080000BC080000BC0800002C
:1000C400BC080000BC080000BC080000BC0800001C
:1000D400BC080000BC08000092410000DC410000A4
:1000E400BC080000BC080000BC080000BC080000FC
:1000F400BC080000BC080000BC080000BC080000EC
:1001040000000000BC080000BC080000BC0800009F
:10011400BC08000028420000BC080000BC08000025
:10012400BC080000BC080000BC080000BC080000BB
:10013400BC080000BC080000BC080000BC080000AB
:10014400BC080000BC080000BC080000BC0800009B
:10015400BC080000BC080000BC0800007442000099
:10016400C04200000C430000BC080000BC080000B2
:10017400BC080000BC080000BC080000BC0800006B
:10018400BC080000BC080000BC080000BC0800005B
:10019400BC080000BC080000BC080000BC0800004B
:1001A400000000000000000000000000000000004B
:0C01B4000000000000000000000000003F
:10020000130181F806C216C41AC61EC822CA26CC1B
:100210002ACE2ED032D236D43AD63ED842DA46DC76
:100220004ADECEC0D2C2D6C4DAC6DEC8E2CAE6CC46
:10023000EACEEED0F2D2F6D4FAD6FED8F3220030CF
:1002400096DA9702002083A2220023A02200F32541
:1002500010342EC09305000273A0458003A1818154
:10026000EF20B00817030020032303FE032103003F
:10027000824273901234D652739002309240A2425E
:100280003243C2435244E244724582551256A2564A
:100290003257C2575258E25872598649164AA64AEE
:1002A000364BC64B564CE64C764D865D165EA65ECA
:1002B000365FC65F13018107730020301300000012
:1002C00013000000130000001300000013000000E2
:1002D00013000000130000001300000013000000D2
:1002E00013000000130000001300000013000000C2
:1002F00013000000130000001300000013000000B2
:1003000083A28181938202E073900234170100205E
:10031000032181F3024182403243C2435244E2440A
:10032000724582551256A2563257C2575258E25859
:1003300072598649164AA64A364BC64B564CE64C6D
:10034000764D865D165EA65E365FC65FD652A1020A
:1003500073900230A24213018107828013000000D3
:100360001300000013000000130000001300000041
:100370001300000013000000130000001300000031
:100380001300000013000000130000001300000021
:100390001300000013000000130000001300000011
:1003A0001300000013000000130000001300000001
:1003B00013000000130000001300000013000000F1
:1003C00013000000130000001300000013000000E1
:1003D00013000000130000001300000013000000D1
:1003E00013000000130000001300000013000000C1
:1003F00013000000130000001300000013000000B1
:10040000F322003093F272FF130380781203B3E2F9
:100410006200711523205500130585FA10C12115BE
:10042000232005009302000063870200711523203A
:100430000500FD12D5BF71150CC1828000000000BF
:1004400000000000000000000000000000000000AC
:10045000000000000000000000000000000000009C
:10046000000000000000000000000000000000008C
:10047000000000000000000000000000000000007C
:10048000000000000000000000000000000000006C
:10049000000000000000000000000000000000005C
:1004A000000000000000000000000000000000004C
:1004B000000000000000000000000000000000003C
:1004C000000000000000000000000000000000002C
:1004D000000000000000000000000000000000001C
:1004E000000000000000397101436EC619A0397187
:1004F00041536AC866CA62CC5ECE19A039710153F5
:100500005AD056D252D44ED64AD826DA22DC06DE4B
:1005100033016140828241114AC026C222C406C60C
:100520008282B24D4101024D924C224CB24B4101AC
:10053000024B924A224AB249410102499244224462
:10054000B240410182803D432A876373C30293779F
:10055000F700BDEFADE5937606FF3D8ABA960CC372
:100560004CC30CC74CC74107E36BD7FE11E2828036
:10057000B306C3408A069702000096966780A600DD
:100580002307B700A306B7002306B700A305B700EB
:100590002305B700A304B7002304B700A303B700E3
:1005A0002303B700A302B7002302B700A301B700DB
:1005B0002301B700A300B7002300B700828093F5A2
:1005C000F50F93968500D58D93960501D58D61B76E
:1005D000939627009702000096968682E78086FA17
:1005E0009680C1171D8F3E96E374C3F8A5B701A08E
:1005F000EF30E000AA8537850000130505F1EF60B4
:10060000C06BEF302000AA85378500001305C5F1C7
:10061000EF60A06AEF20707FAA8537850000130580
:10062000C5F2EF60806901A0EFF2FFEE0945EF002F
:10063000D00AB12AEF20D069716513050520EF209B
:10064000F06FB707002083A507203785000013054A
:1006500085F3EF608066ED23AA85378500001305DA
:1006600085F4EF608065B7850000378500009385CD
:1006700085F5130505F6EF604064EF50E01537840B
:100680000000130504F8EF6080741305803EEF202E
:100690005067C5BFB71702409843B706FFF0411136
:1006A0001367170098C3D84337060200758FD8C365
:1006B0009843B706F7FEFD16758F98C39843B706A3
:1006C000FCFFFD16758F98C3D843B70601FFFD16D2
:1006D000758FD8C39843B70600ECFD16758F98C385
:1006E0003707FF0098C723A6070202C402C6984333
:1006F000C166558F98C3B716024005679C42F18FBB
:100700003EC6A24785073EC4B24781E7A247E397AA
:10071000E7FEB71702409C431397E70063570706AD
:1007200085473EC632478547631FF704B717024027
:10073000D843B706C1FFFD16D8C3D843D8C3D843A2
:1007400013670740D8C3D843758FD8C3D843B706BB
:100750001100558FD8C39843B7060001558F98C331
:10076000984393166700E3DD06FED843B7160240B0
:10077000719BD8C3D84313672700D8C32147DC42F5
:10078000B18BE39EE7FE4101828002C661BFB716CE
:100790000240D842B70700201146318B93870720CB
:1007A0006305C70021466308C70237177A0013079D
:1007B000072098C337170240584311839376F700F8
:1007C0003707002013070700369714239843335741
:1007D000D70098C38280D842D442416649833D8B7A
:1007E000F18E1306270015CF3D47630FE602414700
:1007F000630FE602454781456313E6004146A1E2E7
:100800003747024003270780418B0DC737177A000F
:10081000130707203306C70290C3C9DD9843058339
:1008200049BF81454946E1BF85453546C9BF814538
:100830003D46F1B737173D0013070790E1BF371565
:10084000024058559316F700585563DF060411838C
:100850003D8B9306170037177A001307072033578D
:10086000D70298C35455A182BD8A8DE295463307BD
:10087000D702058398C337170240585794433D8BDE
:10088000050733D7E60298C3984369B705456394D3
:10089000A600E546E9BF3D456396A600D1463387ED
:1008A000E602C9BF8906E5BF3D8B930617003717DF
:1008B0007A00130707203357D702F1B701A0970139
:1008C000002093812114177100201301A173178553
:1008D00000001305A5AB97F5FF1F9385A57213863E
:1008E000018263FAC5008322050023A0550011058B
:1008F0009105E3EAC5FE170500201305A59297753B
:1009000000209385A5C26377B5002320050011055B
:10091000E36DB5FEFD42739002BCFD4273904280D0
:10092000B7820000938202807390023097F2FFFF3B
:100930009382826D93E2320073905230EFF09FD534
:1009400097020000938282CE73901234730020309D
:10095000EFF27FBCB727014093870740631BF50088
:100960008545130500204D2F8145130500206D2777
:10097000E9B6B737014093870780E31BF5FE85454D
:1009800013050040512F814513050040CDB75C4150
:100990003707F1E01307F7EF944D7D8F9C41D58F1A
:1009A000D44DD58FD441A206D58FD98F5CC11C45BB
:1009B00037F7F1FF1307D77FD4457D8F9C49D58F3B
:1009C00094458606D58FD98F1CC55C55370710FF17
:1009D0007D177D8FDC29FD1793F7F70FD207D98F8D
:1009E0005CD582801C4589C593E717001CC58280B1
:1009F000F99BEDBF1C4589C593E707101CC5828094
:100A000093F7F7EFE5BF1C4593E787001CC582808D
:100A100008450D81058982801C4593E747001CC568
:100A2000828008450981058982801C4591C5370768
:100A30005000D98F1CC582803707B0FF7D17F98F12
:100A4000D5BFA54763F7B7048D47138765FF330705
:100A5000F7020328C5009D47B397E70093C7F7FF48
:100A6000B3F70701B396E600DD8E54C5994763E3FB
:100A7000C70495477D163306F6025859FD47B397CC
:100A8000C70093C7F7FFF98F3396C5005D8E50D925
:100A900082800D473387E502032805019D47B39700
:100AA000E70093C7F7FFB3F70701B396E600DD8EC3
:100AB00014C96DBFB14763E2C70295476516330697
:100AC000F6021859FD47B397C70093C7F7FFF98F90
:100AD0003396C5005D8E10D9828095474D1633063A
:100AE000F6025855FD47B397C70093C7F7FFF98F34
:100AF000B395C500DD8D4CD582805C4191C537072B
:100B00000004D98F5CC18280370700FC7D17F98F04
:100B1000D5BFEFF25FA001112A8423040100A54490
:100B20001C8463F8F40423040100A54621461C84B8
:100B300063FCF606231501002304010095461C847E
:100B400063FEF60C38853C8599460D46B3F7D7020F
:100B5000056513050580B3D7C7023357D702BA9787
:100B6000C207C1837C853C8505611D8D4205418599
:100B7000E9B21C4493E787001CC42285513D75FDF2
:100B80001C4493E747001CC42285613D75FD7844F1
:100B90001C8414108607B6972396E7FE1C848507ED
:100BA00093F7F70F5C84ADBFA30401009C846378C6
:100BB000F6001C84850793F7F70F5C848DBF98843B
:100BC0009C840C100607850786072E97AE9703575F
:100BD000C7FE83D7C7FE63FDE7029C848607AE97F6
:100BE00083D7C7FE7C859C84988485078607AE974B
:100BF00083D5C7FE931717001810BA972396B7FE30
:100C00009C8438850C1085078607AE972396E7FEEF
:100C10009C84850793F7F70FDC8449BF1C84101070
:100C2000388589078607B29783D7C7FEBA97C20768
:100C3000C1837C851C84850793F7F70F5C8401B71B
:100C4000B7F7FF1F03A5477082801C4141677917E2
:100C5000F98F1CC123200500232205002324050051
:100C6000B707024023260500138787006317E500B6
:100C7000D8431367F700D8C382801387C701631670
:100C8000E500D8431367070FFDB713870703631801
:100C9000E500D8438566938606F0558FE9BF138734
:100CA00047046315E500D843BD66C5BF13878705B4
:100CB0006316E500D843B7060F00C5B71387C7060C
:100CC0006316E500D843B706F000C1BF13870708D5
:100CD0006316E500D843B706000FC1B713878740F6
:100CE0006319E50003A747401367F70023A2E74015
:100CF00082801387C7416317E50003A74740136746
:100D0000070FEDB793870743631BF500B707024052
:100D100003A747408566938606F0558FC1BFB70786
:100D20000240138747446316E50003A74740BD66AA
:100D3000EDB7138787456317E50003A74740B7065C
:100D40000F00E1BF1387C7466317E50003A74740BD
:100D5000B706F000D9B7138707486317E50003A764
:100D60004740B706000F55BF138707496319E500D1
:100D700003A7474D1367F70023AAE74C8280138728
:100D8000074A6317E50003A7474D1367070FEDB741
:100D90001387074B6319E50003A7474D85669386C4
:100DA00006F0558FD1BF1387074CE319E5FC03A765
:100DB000474DBD66FDB71C4161773D0794517D8F5E
:100DC0009C45D58F9449D58FD449D58F944DD58FD7
:100DD000D44DD58FD451D58F9455D58FD98F1CC173
:100DE000DC455CC19C411CC5DC415CC582801C416A
:100DF00089C593E717001CC1828041677917F98F75
:100E0000DDBF9C4513F7070113F8F70001C7D84170
:100E10003368E8008E2113F7F50F39C31841814676
:100E2000854E3D4F930F800293028004214E3396EE
:100E3000DE00B3F8C5006311160393982600331340
:100E40001F011343F3FF3377E300B318180133E7AF
:100E5000E800639FF70550C98506E39AC6FD18C1EF
:100E60001307F00F6375B70454412146854E3D4F7B
:100E7000930F800293028004414EB398CE0033F763
:100E800015016392E8021317260001173313EF00D0
:100E90001343F3FFB376D3003317E800D98E639D75
:100EA000F701232A15010506E319C6FD54C1828006
:100EB000E39457FA10C94DB7E39757FE232815015D
:100EC000DDB748456D8D3335A00082800CC9828026
:100ED00019C20CC982804CC98280B707002023A0A8
:100EE000A7228280B707002003A707228947102185
:100EF0006311F70214318D4763EDD7003C219A0648
:100F000037E700E09607D58F93F7F70F3297230066
:100F1000F74054410547935756003317C70089CA15
:100F2000938707048A07B7E600E0B69798C38280E4
:100F300093870706C5BFB7160240DC4251777D177D
:100F4000F98F5D8DC8C28280371702405C4391469D
:100F5000B18B6385D700A1466382D706B7177A00A5
:100F6000938707201CC1371602405C4237070020D8
:100F7000130707019183BD8BBA9794231C41B3D704
:100F8000D7005CC15442A1829D8ABA969422B3D6FE
:100F9000D70014C55442AD829D8A36971823B3D723
:100FA000E7005CC558423983937637001387418048
:100FB00036971823B3D7E7021CC982805C43584395
:100FC000C166C983758FB7F6FF1F83A6C670BD8B38
:100FD00089071396160163480600C54601466392C9
:100FE000D702C94739A88946638FD702BD46638EA9
:100FF000D702C146638ED702C54601466393D70028
:10100000C1471DEF3747024003270780418B05C7C3
:1010100037177A0013070720B307F7021CC121D640
:101020001C41858381B701466DBF0546B547D1BFD9
:101030000146BD47F9B737173D0013070790E9BFD1
:10104000B7150240D8559316F700D85563DF06044C
:1010500011833D8B9306170037177A00130707207B
:101060003357D70218C1D455A182BD8A8DE2954667
:101070003307D702058318C1371702405857144168
:101080003D8B050733D7E60218C1184171B7854576
:101090006394B600E546E9BFBD456396B600D14608
:1010A0003387E602C9BF8906E5BF3D8B930617006B
:1010B00037177A00130707203357D702F1B799C5BE
:1010C000371702405C4B5D8D48CB8280B7170240DA
:1010D000D84B1345F5FF798DC8CB828099C537175A
:1010E00002401C4F5D8D08CF8280B7170240984F99
:1010F0001345F5FF798D88CF828099C53717024057
:101100005C4F5D8D48CF8280B7170240D84F1345A2
:10111000F5FF798DC8CF828099C5371702405C47AB
:101120005D8D48C78280B7170240D8471345F5FF49
:10113000798DC8C782801A218D6793870704B621ED
:101140007D8F9E21D58FD621D58FF621D58F9625DF
:10115000D58FB625D58FD625D58FF625D58FD98FA6
:101160001EA15A2DFD779387F77FF98F5EAD9E29DB
:101170001EA982801E2189C593E707041EA18280D3
:10118000C207C18393F7F7FBC207C183C5BF4EA552
:1011900082804A2582800A256D8D3335A0008280A9
:1011A000EFF26FB71629F577FD17F58FF621DA25DF
:1011B0007971D58F1EA95625FD779387379FF58FB7
:1011C000D6212A842EC6D58F9625D58FB625D58FC4
:1011D0005EA55E29C207C18393F7F7CFD98F5EA9B9
:1011E00068089D33B747014093870780B245631E67
:1011F000F402A2576547B387E70298419306400679
:101200000A07B3D7E70233D7D702B3F7D7021207DB
:10121000920793872703B3D7D702BD8BD98FC20715
:10122000C1831EA445616FF04FB19257E1B791C5DC
:101230005E250967D98F5EA582805A25F977FD174B
:10124000F98FD5BF13F7F50F85471583B395B70011
:101250006319F7009307C500984301CED98D8CC35D
:101260008280894693074501E318D7FE930705015D
:10127000E5B793C5F5FFF98DDDB793F5F51F4EA1E1
:1012800082804A211375F51F82800A216D8D3335C6
:10129000A000828013F7F50F85461583B397B6003B
:1012A0006311D7025A25F98F1A210145420741835C
:1012B00081CB0545A181B315B5006D8F3335E000B5
:1012C000828089466314D7001A29F1BF5A29E1BFE9
:1012D000B70700209387C7239843636FA702D043C3
:1012E000B386C7006316D50054413E85B296D4C379
:1012F0005041B306C500631CD700B706002083A683
:1013000046226306D70054431843B29654C118C10D
:101310006303F50088C38280BA877DBFEFF20F9E1A
:1013200041112AC6EF10C035B706002083A7462218
:101330003706002093864622130686223245A1EF07
:10134000370700209307873893F5F700130787388E
:1013500081C51387F700419BB70500209385C523FE
:1013600023A2050098C19965C115AE97C19B23A220
:10137000070023A00700B385E7409CC21CC3B70742
:10138000002023A8B722B707002023A6B722B7075B
:1013900000804CC31CC2032A0600B377AA0085E371
:1013A0009307F5FF3957636CF7009307050113F7AF
:1013B000F70041C313F707FF410763EBE7068144DA
:1013C00089A022872E8461A058C15CC01137584083
:1013D000B7060020938606239042B307E94023A076
:1013E000F90063F3C7009CC2B70700203367EA0027
:1013F0009387472358C09843C1042320040005075E
:1014000098C3EF10E04493F7F400D1CBA167938722
:101410000780739007303786000037850000130679
:1014200086F993050011130505FCEF50100901A082
:10143000BA87370700200329C7229309C722E36030
:10144000F9F8370700200324C7231307C7235040A8
:101450006374F6000C40B5F59442E38286F61440BE
:10146000044314C33307F64093060002E3F1E6F6A3
:101470003305F4009376F500A1DAA167938707801E
:10148000739007303786000037850000130686F911
:101490009305F00C130505FCEF50300201A02685E2
:1014A00041016FF0EF8855C1EFF2EF86B7070020DA
:1014B000032745FF83A787222A84B376F7009DE29E
:1014C000A1679387078073900730378600003785C0
:1014D0000000130686F993054012130505FCEF5032
:1014E000C07D01A0832605FF9DC2A1679387078069
:1014F000739007303786000037850000130686F9A1
:1015000093055012130505FCEF50207B01A093C7F3
:10151000F7FFF98F232AF5FEEF108016B70700209A
:101520009387C7229443032744FF130504FF36978C
:1015300098C3793BB7070020938787239843050713
:1015400098C3EF10E0306FE05FFF8280B7070020A4
:1015500003A5C7228280B7E700E041572387E74011
:101560002386E740B7F700E023A0070023A2070087
:10157000814694C70147D8C7370700208325072035
:101580001307401F814633D6E5023D4790CBD4CBAD
:1015900098C38280EFE23FF8411102C6F327503032
:1015A0003EC6B2470D478D8B6384E702A1679387E0
:1015B00007807390073037860000378500001306D8
:1015C00046FE9305600B130505FCEF50006F01A06C
:1015D000B787002093870700BD8B9DC3A1679387C2
:1015E00007807390073037860000378500001306A8
:1015F00046FE9305B00B130505FCEF50006C01A0EF
:10160000993FB7E700E0056723A0E710116723A023
:10161000E71023A40180EFE0BFCE014541016FE058
:10162000DFF173110134A16793870780739007304E
:10163000B7F700E023A20700EF10C00611C5B7E717
:1016400000E0116723A0E720A16793878788739044
:1016500007307311013473002030A167938707802E
:1016600073900730938781809843050798C38280E1
:10167000138781801C438DE7EFE2FFE9A167938721
:101680000780739007303786000037850000130607
:1016900046FE93052010130505FCEF50006201A0E3
:1016A000FD171CC391E7A167938787887390073064
:1016B00082802165130505807315053082807310C3
:1016C00005308280930785007D575CC118C55CC5D5
:1016D0001CC92320050082802328050082809841B0
:1016E000FD5693078500631ED7001C49D843D8C117
:1016F0000CC79CC5CCC31C4188C985071CC182800E
:10170000B687D4439042E37DC7FECDB75441184518
:101710001C4998C654C3D4436393A600D8C39843C6
:10172000232805007D1798C388438280EFE2BFDE3F
:1017300041112AC61D373245005D1D3F1335140087
:1017400041016FE09FDFEFE21FDD32893041045D30
:101750002A8409EE1C41014591E70844EF106078A6
:1017600023240400850404DC6FE03FDD63100902DC
:101770004841EF5060495C4038400145BA971844F1
:101780005CC0E3E1E7FE1C405CC0E9BF4845EF50A8
:10179000A0473C4058441440B307F0403E9758C41B
:1017A0006375D7001844BA975CC489470145E31BA9
:1017B000F9FACDD8FD147DB7EFE25FD42045411191
:1017C0002AC605E4A16793870780739007303786A0
:1017D00000008565378500001306C600938555BD5A
:1017E000130505FCEF50604D01A0185C5C5C63655F
:1017F000F702A16793870780739007303786000050
:101800008565378500001306C600938565BD130501
:1018100005FCEF50804A01A0185C01496378F7028B
:101820008344540401466C002285313F939984011E
:1018300093D98941FD572A89639EF9005C5099C765
:1018400013054402EF10E03F11C105494A854101EB
:101850006FE01FCE9307F0076395F902A1679387A6
:101860000780739007303786000085653785000054
:101870001306C600938565BF130505FCEF50E043D2
:1018800001A08504E204E184A3029404C1B73041BD
:1018900015C2EFE25FC858451445AA87329758C56C
:1018A0006364D700184158C52E85CC47EF50C0352A
:1018B0006FE0BFC88280EFE21FC62A84793B834471
:1018C000540413094402E204E18463459002FD5785
:1018D000A302F404713B513383444404130904010B
:1018E000E204E18463499002FD572302F404493382
:1018F0006FE0BFC43C4491CB22857D3D19C1EF1000
:10190000E050FD14E204E184C9B75C50E9D34A8594
:10191000EF102033E5B71C48E1DB4A85EF10603259
:1019200019C1EF10A04EFD14E204E18465BFEFE29F
:101930009FBE41111DE1A167938707807390073017
:1019400037860000378500001306C6009305001196
:10195000130505FCEF50603601A05C5D2EC62A849D
:10196000BDC33841B3B7E702B9EFC5393040585C61
:101970001440232C0402B307E602B24554C0338757
:10198000F600918FB6975CC4FD572302F40418C487
:10199000A302F40495E11C4899CB13050401EF1050
:1019A000402A11C5B7E700E0116723A0E720C9313D
:1019B000054541016FE07FB813050401213313058C
:1019C00044020933EDB7A16793870780739007300E
:1019D00037860000378500001306C60093055014B3
:1019E000130505FCEF50602D01A0EFE2DFB24111BD
:1019F00039C1B3B7A502AA849DEF3305B502930799
:101A000030FB63EAA7021305C5042EC6EFF01F9151
:101A10002A8411CDB245AA8799C19307C5042CC069
:101A20001CC044DC85452285193723240404228503
:101A300041016FE09FB0A1679387078073900730E3
:101A400037860000378500001306C6009305601C2A
:101A5000130505FCEF50602601A0EFE25FA901111C
:101A600032C61DE1A16793870780739007303786E0
:101A70000000378500001306C6009305E032130509
:101A800005FCEF50802301A02A842E89B6848DE5C1
:101A90003C419DC3A16793870780739007303786C9
:101AA0000000378500001306C6009305F0321305C9
:101AB00005FCEF50802001A089476398F402585C30
:101AC00085476304F702A167938707807390073007
:101AD00037860000378500001306C60093050033E3
:101AE000130505FCEF50601D01A0EF10E03215E575
:101AF000B247014C85C7A167938707807390073071
:101B000037860000378500001306C6009305303382
:101B1000130505FCEF50601A01A0014C094BFD595B
:101B2000930B040137EA00E0916AA5A85C50C5C395
:101B300013054402EF10E01059A8B24781E70D3EAB
:101B4000014571A863150C002808EF10401E0D36E2
:101B5000EF001033193683474404E207E1876394AA
:101B600037012302040483475404E207E1876394A6
:101B70003701A3020404ED3C6C002808EF10801C20
:101B80003DE9E13C185C5C5C631EF704D534B2456A
:101B90005E85EF00307F2285393BEF00704B29C90D
:101BA000054C653C185C5C5C6364F700E39764F982
:101BB0002686CA8522858329840371363C44BDD795
:101BC00089476394F400639A09002285F53611C5AC
:101BD000B7E700E0116723A0E720593C0545056100
:101BE0006FE07F9471342285F931EF0070464DBF6C
:101BF00023205A2175B722857D39EF00704589B7BA
:101C0000EFE2DF8F41111DE1A16793870780739099
:101C1000073037860000378500001306C60093059D
:101C20002040130505FCEF50400901A02A84328AA8
:101C300036898DE53C419DC3A167938707807390EA
:101C4000073037860000378500001306C60093056D
:101C50003040130505FCEF50400601A0894763188A
:101C6000F902585C85476304F702A16793870780F0
:101C70007390073037860000378500001306C600D2
:101C800093054040130505FCEF50200301A02EC62C
:101C9000EFF03FA2185C5C5CAA8AB2456366F7006D
:101CA000894781446318F902834454044A86228593
:101CB00093998401032B8403793493D98941FD5787
:101CC0006391F9043C449DC78947631CF900630A8A
:101CD0000B0085445685EFF09F9E268541016FE0FD
:101CE0003F852285D13C75D5E3050AFE8547232033
:101CF000FA00C5B75C50F1DF13054402EF007074C1
:101D0000DDB79307F0076394F902A1679387078013
:101D10007390073037860000378500001306C60031
:101D20009305D048130505FCEF40307901A08504E8
:101D3000E204E184A302940469BFEFE2CFFD1DE158
:101D4000A167938707807390073037860000378537
:101D500000001306C6009305D04A130505FCEF40AA
:101D6000D07501A03C412A849DC3A1679387078059
:101D70007390073037860000378500001306C600D1
:101D80009305104B130505FCEF40307301A01C4177
:101D9000AE848DE71C459DC3A16793870780739030
:101DA000073037860000378500001306C60093050C
:101DB000604B130505FCEF40507001A0EFF07F8FE2
:101DC000185C5C5C2A896370F70883475404050734
:101DD00018DC93968701E1867D57639AE6023C44BE
:101DE00085C32285EFF05F9D01E905444A85EFF048
:101DF0001F8D22856FE06FF4EDD885479CC0F5B745
:101E00005C50E5D713054402EF00B063F1BF130740
:101E1000F0076394E602A167938707807390073009
:101E200037860000378500001306C600930550531F
:101E3000130505FCEF40706801A08507E207E18704
:101E4000A302F4045DB7014455B7EFE24FEA011174
:101E500032C61DE1A16793870780739007303786EC
:101E60000000378500001306C600930510551305C2
:101E700005FCEF40906401A02A84AE898DE53C41C9
:101E80009DC3A16793870780739007303786000052
:101E9000378500001306C60093055055130505FC51
:101EA000EF40B06101A0EF00307715E5B24701497E
:101EB00085C7A16793870780739007303786000036
:101EC000378500001306C6009305A055130505FCD1
:101ED000EF40B05E01A001497D5A930A440237EBFE
:101EE00000E0916B95A8B24789E7EFF06FF80145E4
:101EF00069A8631509002808EF007063EFF04FF739
:101F0000EF000078EFF06FF583474404E207E187C4
:101F1000639447012302040483475404E207E187E2
:101F200063944701A3020404EFF08FF46C002808C7
:101F3000EF00506125E52285EFF04FFF31C9B24532
:101F40005685EF0030442285EFF0FF96EF005010E9
:101F500019E123207B210549EFF02FF0045CC1D467
:101F6000CE852285FD14EFF09F9204DC1C4899CBAE
:101F700013050401EF00F04C11C5B7E700E011674D
:101F800023A0E720EFF0CFEE054505616FE0AFD964
:101F90002285EFF05F92EF00B00B75BF2285EFF066
:101FA0009F91EF00F00A2285EFF04FF84DD581B7F1
:101FB000EFE2CFD401112EC61DE1A1679387078000
:101FC0007390073037860000378500001306C6007F
:101FD0009305305E130505FCEF40304E01A03C41F7
:101FE0002A849DC3A1679387078073900730378643
:101FF0000000378500001306C6009305705E1305C8
:1020000005FCEF40904B01A0EF0010610DE5B247D9
:102010009DC3A167938707807390073037860000C0
:10202000378500001306C6009305C05E130505FC46
:10203000EF40B04801A081440149FD59130A440210
:10204000B7EA00E0116B6DA0B2479DE79DC0A167A4
:10205000938707807390073037860000378500002C
:102060001306C60093052063130505FCEF40F044FA
:1020700001A0EFF0EFDF7DA0631509002808EF0055
:10208000104BEFF0EFDEED2BEFF02FDD8347440434
:10209000E207E18763943701230204048347540471
:1020A000E207E18763943701A3020404EFF04FDCF9
:1020B0006C002808EF00104941E12285EFF00FE79E
:1020C00035C51C4089EBEFF04FD90844EF0090561E
:1020D000AA84EFF0EFD9B2455285EF00B02A2285ED
:1020E000EFF06FFDEF00C07619E123A06A210549EA
:1020F000EFF0AFD61C5CA9DBFD171CDC1C4081E7B0
:10210000EF00307908C41C4899CB13050401EF0097
:10211000503311C5B7E700E0116723A0E720EFF0C7
:102120002FD58544268505616FE08FC02285EFF0AD
:102130008FF8EF00E07165BF2285EFF0CFF7EF0079
:1021400020712285EFF08FDE5DD1E9DCEFF0EFD07A
:102150005C50814589C71C58A9459C439D8D084406
:102160008144EF00B064EFF0AFD06DBFEFE2AFBAE3
:1021700041111DE1A167938707807390073037866F
:102180000000378500001306C6009305407F130545
:1021900005FCEF40903201A02A84EFF00FCC1C5CCC
:1021A000485C1D8D2AC6EFF0AFCC324541016FE08F
:1021B000CFB815E5EFE22FB6A1679387078073903C
:1021C0000730378600008565378500001306C60096
:1021D000938585AC130505FCEF40302E01A09DCD05
:1021E00037660020930686388147014713068638F4
:1021F000214883A846006398A80093173700B29738
:102200008CC3C8C321A891E783A806006393080084
:10221000B6870507A106E31E07FDFDF38280EFE206
:102220008FAF41112A842EC632C4EFF00FC383470B
:1022300044047D572246E207E187B2456394E700F4
:1022400023020404834754047D57E207E187639423
:10225000E700A302040432C62EC4EFF06FC11C5C79
:10226000A245324689E713054402EF003016228565
:10227000EFF06FE441016FE04FACEFE2CFA9014610
:102280009145EFF08FF66FE04FABEFE2CFA8411131
:102290002AC62EC4EFF06FBC3245A24501443C452E
:1022A00091E71C5D014499E32CC50544EFF04FBC58
:1022B000228541016FE06FA8EFE2EFA541112E8664
:1022C0006C0002C6EFF07FB8324541016FE0EFA627
:1022D00037070020130787241C439443B7070020C7
:1022E0009387872681E67D5798C382801843584795
:1022F0001843DDBFEFE28FA037090020B7070020A9
:102300009304492483A987272A849C40884041114B
:10231000A388070411052EC6EFF04FBF7D57930722
:102320004924B245631CE40295C9B767002093872E
:10233000C74C9440D84398C610479440D0C69440A8
:102340001047910654C29440910614C798405CCB44
:102350009843050798C341016FE08F9D98434E94C1
:1023600040C3637B3401370700200325C7248C4317
:102370009105EFF0CFB6C5B73707002003258724B6
:102380008C439105EFF0AFB5B70700209387872600
:102390009843E372E4FC80C37DBFEFE22F9637647D
:1023A0000020B70900201304044E370A002093844C
:1023B00049259C40EDDFEFF04FAA5C4403A9C7001C
:1023C00013054900EFF08FB413070A251C43FD17CE
:1023D0001CC39C40FD179CC0EFF08FA90325090387
:1023E000EFF06F8C4A85EFF00F8CD1B7EFE22F90B2
:1023F00013192600AA8A4A852E8A368BBA8BBE8983
:10240000EFE0DFF11DC1AA8413054005EFE01FF1E5
:102410002A8409C904D98147C146631A0A00230ADC
:10242000050225A02685EFF00F887D5565A23307AC
:10243000FA00030707003306F400230AE60201C787
:102440008507E396D7FEA3010404A54763F4770349
:10245000A167938707807390073037860000378520
:1024600000001306060293057039130505FCEF40C2
:10247000D00401A0130A44005285232674032322AA
:10248000740523240404EFF02FA513058401EFF055
:10249000AFA429471305C9FF33077741269500C824
:1024A00018CC40D023060404A30604042307040424
:1024B000A307040423080404A30804045A86D68549
:1024C0004199EFD0FFF308C06384090023A089007D
:1024D000EFF0AF98B7070020938707259843B7041C
:1024E0000020B7690020050798C3138744241843C8
:1024F000938444241389893C6310070E80C0984359
:1025000085476316F7069389893C930A890C4E85A3
:10251000D109EFF02F9BE39C3AFF37650020930A27
:10252000054913050549EFF0EF9937650020930938
:10253000454A1305454AEFF0EF983765002013052B
:10254000854BEFF02F98376500201305054EEFF00F
:102550006F97376500201305C54CEFF0AF96B707AE
:10256000002023A45725B707002023A63725B70747
:1025700000209387C7259843050798C33707002095
:10258000130707265C54144363F3F6001CC351473A
:10259000B387E702CA97D843144718C454C41447F2
:1025A00023A246012324470198435CC8050798C32A
:1025B000EFF00F8CB707002083A74727054599CB7D
:1025C0009C40D8575C546377F700B7E700E0116789
:1025D00023A0E7206FD03FF5B707002083A7472748
:1025E000D9F79C40D8575C54E3E3E7F880C041B783
:1025F000EFD27FF2B7070020B78500003725000033
:1026000093874726014781461306001093854503AB
:102610001305A539E13B0544631E8502EF007056A2
:10262000631A8502A1679387078073900730B70705
:1026300000207D5723A4E726B707002023AAA7265A
:10264000B707002023AC0726EFE0DFF483A7C180A3
:102650006FD0BFEEFD57E31BF5FEA16793870780A0
:1026600073900730378600008565378500001306B4
:10267000060293850584130505FCEF40006401A064
:10268000B7070020938787259843050798C3828062
:10269000B707002003A587278280B707002003A57E
:1026A00087278280B707002083A7872563990718AB
:1026B000EFD27FE6B7070020938787278043050482
:1026C00080C321ECB70700209387872498431843E1
:1026D00005C7A1679387078073900730378600008E
:1026E00085653785000013060602938575AC1305D2
:1026F00005FCEF40805C01A0370700201307C724CA
:102700009443104390C3B707002014C39387C72690
:102710009843050798C3EFF0BFBB37060020930727
:1027200086269C4337670020B705002013068626BF
:102730001307873C9385452401456375F4029C414A
:10274000D146DC57B387D7023E971843854763F3DA
:10275000E7000545B707002083A7C72791C30545B4
:102760006FD0BFDD370E0020B70E0020514F93070A
:102770008E249443944281E6FD571CC2C9B79C4302
:10278000DC47DC47D4436374D40014C24DBF83A834
:10279000870003A8C700D44B1383470023A4080174
:1027A0002322180183A846006394680023A206012F
:1027B00003A8060023AA07007D1823A0060194574A
:1027C00095CA03A8C70183A8070283AF4600232444
:1027D000180183A8070223A20801138887016394C4
:1027E0000F0123A2160103A8060023A407027D18E7
:1027F00023A0060193860E2603A8C70283A806001D
:1028000063F4080123A00601B306E803BA9683A87F
:10281000460083AF880023A4170123A6F70183AFE6
:10282000880023A26F0023A46800D4CB9C428507B4
:102830009CC29C41DC57E36CF8F205450DBFB7071D
:1028400000209387072798430145050798C3828096
:10285000EFD2DFCA37040020130484251C40411145
:1028600085E7A1679387078073900730378600005C
:10287000856537850000130606029385358B1305A1
:1028800005FCEF40804301A0EFE03FDD1C40FD1759
:102890001CC01C4089CB01452AC6EFE07FDD3245D4
:1028A00041016FD0FFC8B707002083A70725E5D7F0
:1028B000B76600203765002081479386864B370F27
:1028C00000201305853CD14837030020370E002037
:1028D000854E59A8DC46DC47CC4F9053985790C59D
:1028E00003A807022322B800032847009385870125
:1028F0006313B80050C3104323A407027D1610C30E
:102900008C47D047D84B1388470090C54CC24C43E6
:102910006393050150C3104323AA07007D1610C31B
:1029200013070F26D0570C4363F3C50010C33307BA
:1029300016032A974C4383AF85008CC723A6F70163
:1029400083AF850023A20F0123A405010C43D8CB3C
:1029500085050CC313074324184358576366E600E4
:102960001307CE272320D70198422DF799C3EFF004
:102970003F96B707002013870727044313840727D0
:1029800091CC370900208549313B09C59307C927F8
:1029900023A03701FD14EDF823200400B707002021
:1029A00083A7C727E38907EEB7E700E0116723A0F5
:1029B000E7200545D5B5EFD21FB641111DE1A1674E
:1029C00093870780739007303786000037850000B3
:1029D000130606029305104F130505FCEF40E02D8A
:1029E00001A09DE1A1679387078073900730378628
:1029F000000037850000130606029305204F1305DB
:102A000005FCEF40802B01A0B707002083A7872596
:102A10009DC3A167938707807390073037860000B6
:102A200037850000130606029305304F130505FC99
:102A3000EF40A02801A02A842EC6EFF07FC41840E2
:102A4000B245B707002003A58727B307B7001CC00E
:102A50006370E50263E0E7020144DD3B11E5B7E79F
:102A600000E0116723A0E720228541016FD0FFAC71
:102A700063E4E700E372F5FE81453385A740EFF09C
:102A80007F870544D9BF19E5B7E700E0116723A0A8
:102A9000E7208280EFD23FA8B707002083A78725D1
:102AA00041119DC3A16793870780739007303786D4
:102AB00000003785000013060602930590541305A5
:102AC00005FCEF40801F01A02AC6EFF07FBB324516
:102AD0008145EFF03F82AD3B11E5B7E700E01167BC
:102AE00023A0E72041016FD05FA5B707002003A70F
:102AF0008725B70700209387C72701C7054798C3D5
:102B0000828023A00700B7070020138707261843F9
:102B100013860726B76700209387873C5148B30682
:102B20000703B385D700884115C5C841A106BE96E5
:102B30004841C8C16314D5005441D4C1D146B3063D
:102B4000D702B697DC43D447B707002023A2D72487
:102B500018C2828015E7EFD21F9CA1679387078078
:102B600073900730378600008565378500001306AF
:102B70000602938525C0130505FCEF40001401A053
:102B80007D1771BFEFD23F9905E5A1679387078055
:102B9000739007303786000085653785000013067F
:102BA00006029385C5C1130505FCEF40001101A085
:102BB000B70700202E8483A54724E105EFE03FB24C
:102BC00085452285EFF00FF36FD03F97EFD2BF948A
:102BD0002A8705E5A16793870780739007303786BA
:102BE000000085653785000013060602938525C51C
:102BF000130505FCEF40600C01A0B7070020938788
:102C0000472454432E858C4303A88600D4CD8C439F
:102C100023A0050303A807008C46610823A2050131
:102C200003A807009C43610823A4060198D71C430E
:102C300085071CC311C27D55B285EFF0AFEB6FD095
:102C4000DF8F5C45DC4795E7EFD2FF8CA167938768
:102C50000780739007303786000085653785000050
:102C600013060602938525C8130505FCEF40E00412
:102C700001A0D04F945398579385870114C6D0C2B2
:102C800050436313B60054C3144323A40702FD1634
:102C900014C33707002003278725D45725EF8C4717
:102CA000D047D84B90C5D04748434CC29385470086
:102CB0006313B50050C3104323AA07007D1610C349
:102CC000370700201307072610436373D60014C389
:102CD00051473386E602376700201307873C329757
:102CE0005043084690C7C8C708464CC10CC6D8CB4D
:102CF0001C43014585071CC3B707002083A7472451
:102D0000DC5763F8D700B7070020054723AEE72656
:102D100005458280376700201307874B50430846DC
:102D2000D0CF88D308464CC10CC698D7D1B7B707C7
:102D3000002083A7C7261CC1B707002083A78727C9
:102D40005CC18280EFD22FFD411105E5A167938719
:102D5000078073900730378600008565378500004F
:102D6000130606029385D5CF130505FCEF30F074EA
:102D700001A085E5A16793870780739007303786A8
:102D80000000856537850000130606029385E5CFB0
:102D9000130505FCEF30707201A02EC62AC4EFE0C7
:102DA000DF8B37070020B70700201307472483A6CF
:102DB00087271C432245B24583C7170599CB1C437F
:102DC000A38807040544EFE0BF8A228541016FD044
:102DD000CFF69C417D570144E387E7FE370600208C
:102DE0000326C6260328050058416307C80063E58B
:102DF000E60023A00500F9B73386E640E37BF6FE44
:102E0000958FBA979CC12537014475BFB70700203D
:102E1000054723AEE7268280B707002083A7472710
:102E2000054581CBB707002003A58725133515007D
:102E3000060582804DC5EFD26FEC3709002093075D
:102E400049249443585513094924D4566373D70829
:102E50001C4D63C8070083270900D457A947958FE5
:102E60001CCD51463307C702B76700209386873CC5
:102E70009384873C369754496398E6049309450048
:102E80002A844E85EFE09F888327090037070020BA
:102E900013070726DC5714435CD463F3F6001CC306
:102EA0005147B387E702A697D843144718C454C4C0
:102EB000144723A236012324370198435CC8050731
:102EC00098C305456FD0CFE683270900DC575CD552
:102ED000CDBF9C436841DC573335F500E5B701456C
:102EE000828011E50145828001456FD00FE5EFD268
:102EF0008FE2B707002083A747242A846385A702AF
:102F0000A167938707807390073037860000856537
:102F100037850000130606029385F504130505FCAA
:102F2000EF30B05901A0BC4785E7A16793870780C0
:102F300073900730378600008565378500001306DB
:102F4000060293850505130505FCEF30105701A017
:102F500054557841FD173CC5E388E6F8D1F7930452
:102F600045002685EFE08FFA7C4029471D8F18CC5D
:102F7000370700201307072614435CD463F3F600D9
:102F80001CC351473387E702B76700209387873C0C
:102F90000545BA97D843144718C454C41447C4C24B
:102FA00004C798435CC8050798C381B775C1EFD2C1
:102FB0008FD634452A8485E6A1679387078073906E
:102FC0000730378600008565378500001306060246
:102FD0009385F509130505FCEF30304E01A07C41C7
:102FE00063F3B700AE8758546302F70A0546639F40
:102FF000C608B706002083A6462463958602A1670B
:103000009387078073900730378600008565378582
:103010000000130606029385A50B130505FCEF308F
:10302000D04901A0144C5CD463C60600A946B387FE
:10303000F6401CCC51463307C702B7670020938681
:10304000873C9384873C369754486391E604130980
:1030500044004A85EFE08FEB37070020130707266F
:103060005C54144363F3F6001CC35147B387E70273
:10307000A697D843144718C454C4144723A2260162
:103080002324270198435CC8050798C36FD0EFCA73
:103090008280B7070020138747241843938747246B
:1030A00009C79443B8460507B8C688438280EFD263
:1030B0008FC637040020EFE04FDA1304C4281C4009
:1030C000B1E7376500201309454F1305454FEFE081
:1030D0006FDF376500209304855013058550EFE0BE
:1030E0006FDEB707002023A027290146B70700207D
:1030F000C145114523A29728EFE03F8F08C019C5AD
:10310000B785000093850506EFF0AF8AEFE04FD654
:103110006FD0AFC2EFD22FC04CC108C9AA8763627B
:10312000B602184D158E0545637BE6009385470072
:10313000B707002003A54728EFE06FDA01456FD0FD
:10314000CFBF6375D6000545E3FBD5FE93854700E9
:10315000B707002003A50728C5B7EFD2CFBB2A8445
:10316000AE8432890C4CA6864A86A69522855D37A8
:1031700019E16FD08FBC1C4C2285BE941C508297E5
:10318000D5B7EFD24FB9B707002083A70728411161
:10319000AA84DC472EC6C04713054400EFE00FD7D2
:1031A00083474402324613F7470011CBA685228598
:1031B0006D371C502285829741016FD00FB8F99B63
:1031C0002302F402FDB7EFD20FB5370400209306B7
:1031D000042898421C4391EBB707002093874728A7
:1031E000904398C390C26FD04FB55C47FD5588435C
:1031F000493FF1BFEFD2AFAF21694111B70A0020BB
:10320000B7090020370B0020B70B00201309C903B2
:1032100083A70A28984329CBDC47814C03AC0700DD
:10322000EFF00FC6EFF0CFC683A789282A849384D6
:103230008928130ACB28636CF50288C0638F0C02BF
:1032400083A74B2890431336160003250A00B305C5
:103250008C40EFE0DFFCEFF0AFDF11EDB7E700E00F
:10326000116723A0E72001A8854C014C55BFA13F61
:1032700080C0EFF0EFDD214C05A00146E36785FD3E
:10328000EFF00FDDA2856285ED3DF5B79247B245BF
:103290008297824763DD070003250A0001468A857D
:1032A000EFE0BFBA35D582472245E3C107FE22448D
:1032B0005C4895E3EFF0CFBD9C40AA8C6373F500AA
:1032C0001937824723A09401FD17E367FCFC8A07A6
:1032D000CA979C43828713054400EFE02FC3D9BFF0
:1032E000834744020C4C924693E717002302F402F2
:1032F0006686B6952285393D45D18347440213F74A
:10330000470019CB1C4C924566862285BE95B13587
:103310001C502285829749B7F99B2302F402CDBF46
:1033200083474402F99B2302F402BDB7834744025A
:10333000924593E717002302F4020CCC9DE1A167AC
:103340009387078073900730378600003785000029
:103350001306860693059035130505FCEF30F0152E
:1033600001A0E6866686E6952285EFF0BFDA2DB7E6
:103370008347440213F7270055F72285EFE0AF9209
:1033800021BFEFD24F99EFF09FD2B707002083A75C
:10339000C7289DE3A167938707807390073037861E
:1033A000000037850000130686069305901113056B
:1033B00005FCEF30901001A0B7070020B785000092
:1033C00037350000938707292547814613060010EB
:1033D000938505081305451FEFF04F8145DD6FD03C
:1033E000CF95EFD2AF91AA8A13058002AE843289BD
:1033F000368ABA89EFD09FF22A8439C9230205029E
:103400009DE0A1679387078073900730378600009F
:1034100037850000130686069305B016130505FCD4
:10342000EF30B00901A0EFF09FC81305440023203E
:10343000540104CC232E440123203403EFE0CFA910
:10344000630809008347440293E747002302F4021C
:1034500022856FD0EF8DEFD20F8C01111DE1A16796
:103460009387078073900730378600003785000008
:10347000130686069305B018130505FCEF30F0031C
:1034800001A0370400201304C4281C403AC62A882F
:1034900001458DC7B6882EC832CA42CC954663C254
:1034A000B602EFF07F973247894781463A86630339
:1034B000F500014608400C08EFE02FDA05616FD0F7
:1034C000CF87814646860C083E85EFE06FF3FDB757
:1034D000B707002083A7072037177A0013070720B4
:1034E000B3D7E7023707002093F7F70F230BF7282E
:1034F0001307803EB387E70237070020231AF72817
:103500008280B7F700E0D8438146799BD8C337075C
:103510000020035747293306A70290CBD4CB98430A
:103520001367070198C398431367170298C3D843DA
:10353000058B75DF9843799B98C38280EFC2BFFDEE
:103540002A841165011185451105EFD03FB9930714
:1035500000207C82371501408D473EC44C00E14776
:10356000130505803EC6EFD0DF8922C837440140ED
:10357000B70708000C08130504803ECC02CA231EBE
:103580000100EFD0FFC1854513050480EFD03FCA8D
:1035900005616FC09FFAEFC27FF6B7440140AE8964
:1035A0003289014493840480634524014A856FC0B5
:1035B0003FF8930500042685EFD03FCD7DD9B38732
:1035C00089008385070026850504C205C181EFD0E7
:1035D000DFCAD9BF138701811C43B77600209386C9
:1035E00086523E95636BD500B78600209386068091
:1035F00063E5A60008C33E858280FD57EDBF7325B5
:103600001034828073252034828073253034828088
:10361000232605000CC150C12324050005458280E6
:103620005C45544118458507B3E7D702638EE70030
:1036300058451C41BA978CA35C4558418507B3E7B0
:10364000E7025CC5054582807955828018455C4556
:10365000630FF70018451C41BA979C239CA11C4599
:1036600058418507B3E7E7021CC50545828001453F
:103670008280EFC25FEA7971130600028145080873
:10368000EFC07FEC8545114502C202C402C6EFD0EF
:10369000FFA4854513050020EFD05FA41165EFD08E
:1036A0009F89371401408547130504804C007C82B4
:1036B00002C6EFD00FF5C147130504804C007C8291
:1036C00002C6EFD00FF4930700024C0013050480EC
:1036D0007C823724014002C6EFD0AFF213050440CC
:1036E000EFD00FA785473ECA3ECCB7070E003ECEAF
:1036F0000C088D47130504402302F10202C802D0D2
:10370000EFD0EFA8854513050440EFD0AFAE854557
:1037100013050440EFD00FAD814513050440EFD0F1
:10372000CFBD13050440EFD00FAE930404402685AF
:10373000EFD00FAE6DFD1305044037240140EFD0EC
:10374000AFAD930404402685EFD0AFAD6DFD1305FA
:103750000440EFD00FBCB7070020239CA728456189
:103760006FC0BFDDEFC23FDB79711306C002814538
:103770004800EFC05FDD85450545EFD05F94370415
:10378000024013058400EFD04FCCB7270140938748
:10379000C7443EC2B70700209387C7293EC48D4760
:1037A0003EC8930700083ECC930700103ECE930717
:1037B00000403ED0930700023ED24C008D671305B7
:1037C00084003ED402C602CA02D6EFD0CFDE4561E5
:1037D0006FC0BFD6EFC23FD43705024085452105F3
:1037E00037240140EFD0AFE0130504409D46054665
:1037F0008145EFD00FA5130504409D46094691452C
:10380000EFD02FA49D460D46130504409545EFD0FB
:103810004FA3130504408545EFD0CF9D8545130583
:103820000440EFD08FA06FC05FD1EFC23FCD011138
:1038300085453145EFD09F8A85452165EFD0FF8BC7
:1038400037140140E1778D44C1498A85130504800E
:103850007C804EC426C2EFD0CFDA13050480A16568
:10386000EFD0CFE6A14761498A85130504C07C806B
:103870004AC426C2EFD0EFD891478A85130504C009
:10388000231031013EC4EFD0CFD7930700028A85C1
:10389000130504C07C804AC426C2EFD08FD6B70778
:1038A00004013EC6B70702003EC8B70700028507FD
:1038B000374400403ECAA1473ECC6C009D471305EB
:1038C00004C0FC86EFD03F878545130504C0EFD0C8
:1038D0007F8A05616FC0DFC5EFC25FC2B744004099
:1038E0002A891304900C938904C089454E85EFD032
:1038F0009F8A05C9CA85138504C0B7440040EFD02C
:103900001F891304900C138904C085454A85EFD0A4
:103910009F8819CD138504C0EFD0BF871375F50FAD
:1039200031A07D141374F40F69F001456FC05FC0BE
:103930007D141374F40F71F8CDBFEFC2DFBD2A8977
:10394000371501402E8413050580A165B284014618
:10395000EFD00FD80D454937135504011375F50FF6
:10396000A53F135584001375F50FBD371375F40F7C
:10397000A537014493170401C18363EC9700371501
:1039800001400546A16513050580EFD06FD46FC0D7
:10399000DFBA1305F00FEFF03FF4B307890088A3F7
:1039A0000504C9BFEFC23FB74111854513050004A7
:1039B000EFD0CFF2A147372401407C8285473EC437
:1039C0004C00C147130504803EC6EFD08FC30146AB
:1039D00013050480A145EFD0AFCF91474C001305EC
:1039E00004807C82EFD0EFC101461305048091452D
:1039F000EFD00FCE930700084C00130504807C82A3
:103A0000EFD02FC001461305048093050008EFD0C6
:103A10002FCC930700104C00130504807C82EFD05C
:103A20004FBE01461305048093050010EFD04FCA26
:103A3000930700204C00130504807C82EFD06FBCFC
:103A400001461305048093050020EFD06FC893074B
:103A500000404C00130504807C82EFD08FBA0146F1
:103A60001305048093050040EFD08FC685679387C8
:103A700007804C00130504807C828564EFD06FB80A
:103A800001469385048013050480EFD06FC44C0079
:103A9000130504806482EFD0CFB60146130504807D
:103AA0008565EFD0EFC289644C0013050480648201
:103AB000EFD02FB50146130504808965EFD04FC1C3
:103AC00091674C00130504807C82EFD08FB30146D0
:103AD000130504809165EFD0AFBFE1774C0013056B
:103AE00004807C82EFD0EFB1014613050480A1650C
:103AF000EFD00FBE4C00371501406482EFD06FB09D
:103B00000546896537150140EFD08FBC41016FC074
:103B1000DFA2EFC25FA0EFD0AFBB6FC01FA2EFC2AA
:103B20009F9FEFD00FBA6FC05FA1EFC2DF9E372417
:103B3000014013050480014693050002EFD04FB900
:103B400013050480014693050004EFD06FB83714C5
:103B500001401305048001468945EFD06FB7130576
:103B600004C001468545EFD0AFB60146930500106D
:103B700013050440EFD0CFB56FC03F9CEFC2BF9993
:103B800079712A89854513050004EFD02FD5372494
:103B90000140930700028D44FC824C08C147130585
:103BA00004803ECE26CCEFD0CFA505461305048079
:103BB00093050002EFD0CFB185454145EFD00FD23C
:103BC000854513050004EFD04FD38547FC824C0890
:103BD000E1473715014026CC3ECEEFD08FA2894772
:103BE000FC824C08914737150140372400403ECEF7
:103BF000EFD02FA10C10B7070C00130504804AD09A
:103C00003ED402D223160102EFD08FD9930770352C
:103C10007C86680085473EC84487EFD0AFAC13056B
:103C20000480054693055052EFD0CFE105461305B9
:103C3000048093054042EFD0EFE0854513050480F2
:103C4000EFD0EFDE45616FC05F8FEFC2DF8C79711F
:103C50002A89854513050004EFD04FC83724014059
:103C6000930700048D44FC824C08C147130504806F
:103C70003ECE26CCEFD0EF98054613050480930581
:103C80000004EFD0EFA485454145EFD02FC5854511
:103C900013050008EFD06FC69147FC824C08E1473E
:103CA0003715014026CC3ECEEFD0AF95A147FC8220
:103CB0004C08914737150140372400403ECEEFD0E5
:103CC0004F940C10B7070C00130504C04AD03ED423
:103CD00002D223160102EFD0AFCC930780357C8649
:103CE000680085473EC84487EFD0CF9F130504C0C6
:103CF000054693055052EFD0EFD40546130504C096
:103D000093054042EFD00FD48545130504C0EFD092
:103D10000FD245616FC07F82EFC2EFFF79712A89B0
:103D200085451145EFD08FBB3714014089478D443D
:103D3000FC824C08C147130504803ECE26CCEFD050
:103D40004F8C0546130504808945EFD06F98854553
:103D50001145EFD0AFB8854537050200EFD0EFB978
:103D60009147FC824C08E1471305048026CC3ECEE7
:103D7000EFD02F89A147FC824C089147130504809E
:103D80003ECE37440040EFD0CF870C10B7070C0071
:103D9000130504404AD03ED402D223160102EFD0CC
:103DA0002FC0930760337C86680085473EC84487F0
:103DB000EFD04F9313050440054693055052EFD0C2
:103DC0006FC805461305044093054042EFD08FC7E6
:103DD000854513050440EFD08FC545616FC0EFF5F1
:103DE000EFC2CFF17971AA8985452145EFD00FAF98
:103DF0003719014085470D44C1444C08130509C0DB
:103E0000FC8226CE22CCEFC0DFFF0546130509C099
:103E10008545EFD0EF8B85454145EFD02FAC8545EB
:103E200013050010EFD06FADE1474C083715014086
:103E3000E48222CC3ECEEFC0DFFC93070002FC827E
:103E40004C089147371501403ECEEFC09FFB0C1048
:103E5000B7070C00372500404ED03ED402D22316BF
:103E60000102EFD0EFB3930790357C866800854759
:103E70003EC84087EFD00F8705469305505237253F
:103E80000040EFD02FBC0546930540423725004047
:103E9000EFD04FBB854537250040EFD04FB9456186
:103EA0006FC00FE9EFC22FE737140140130504403C
:103EB000014693050020EFD0AF8113050440014671
:103EC00093050040EFD0CF8085650146938505803E
:103ED00013050440EFC0DFFF6FC02FE6EFC20FE213
:103EE00079712A8A854513050002EFD02F9F371478
:103EF000014093070010FC820D49C1474C0813058F
:103F000004403ECE4ACCEFC0DFEF05461305044027
:103F100093050010EFC0DFFB930700204C0813054A
:103F20000440FC82EFC0FFED930900404C081305EC
:103F30000440231A31018564EFC0BFEC4C0813051F
:103F4000044093840480E482EFC0BFEBEFF09FF560
:103F500085452145EFD08F98854537050400EFD082
:103F6000CF99E1474C08130504C0231A31014ACC0C
:103F70003ECEEFC01FE991474C08130504C0E48210
:103F8000375400403ECEEFC0DFE70C10B7070C00FF
:103F90001305048052D03ED402D223160102EFD082
:103FA0002FA0930770137C8685475C876800854740
:103FB0003EC8EFC03FF313050480054693055052F9
:103FC000EFD04FA805461305048093054042EFD07B
:103FD0006FA7854513050480EFD06FA545616FC0BD
:103FE0002FD5EFC24FD337140140130504400146CB
:103FF00093050020EFC0DFED130504400146930553
:104000000040EFC0FFEC85650546938505801305EC
:104010000440EFC0FFEB6FC04FD2EFC2CFCF3714D9
:10402000014013050440014693050020EFC05FEAFC
:1040300013050440054693050040EFC07FE9856500
:1040400001469385058013050440EFC07FE86FC0EB
:10405000CFCEEFC24FCC37140140130504400146C8
:1040600093050020EFC0DFE61305044005469305E5
:104070000040EFC0FFE58565054693850580130583
:104080000440EFC0FFE46FC04FCBEFC2CFC837147E
:10409000014013050440054693050020EFC05FE38F
:1040A00013050440014693050040EFC07FE285659B
:1040B00001469385058013050440EFC07FE16FC082
:1040C000CFC7EFC24FC53714014013050440054662
:1040D00093050020EFC0DFDF130504400146930580
:1040E0000040EFC0FFDE856505469385058013051A
:1040F0000440EFC0FFDD6FC04FC4EFC2CFC1797184
:10410000AA8485454145EFC07FFD85451305000222
:10411000EFC0DFFC854537051000EFC01FFE856747
:104120000D44FC824C08E1473715014022CC3ECEBD
:10413000EFC03FCD914737150140FC824C089147B5
:10414000130505403ECEEFC0DFCBB7070C000C10C7
:10415000375500403ED426D002D223160102EFD0BC
:104160002F8405469305505237550040EFD08F8D70
:10417000930750147C86680085473EC84087EFC08F
:104180007FD6854537550040EFD06F8A45616FC0B7
:10419000CFBA397106DE16DC1ADA1ED82AD62ED42A
:1041A00032D236D03ACE3ECC42CA46C872C676C467
:1041B0007AC27EC0C525F250E2525253C2533255E4
:1041C000A255125682567247E2475248C248324EB2
:1041D000A24E124F824F216173002030397106DEEA
:1041E00016DC1ADA1ED82AD62ED432D236D03ACEDF
:1041F0003ECC42CA46C872C676C47AC27EC0EF00C0
:104200004076F250E2525253C2533255A2551256E2
:1042100082567247E2475248C248324EA24E124F6F
:10422000824F216173002030397106DE16DC1ADA04
:104230001ED82AD62ED432D236D03ACE3ECC42CA5E
:1042400046C872C676C47AC27EC0EF00607EF25065
:10425000E2525253C2533255A255125682567247F9
:10426000E2475248C248324EA24E124F824F21615D
:1042700073002030397106DE16DC1ADA1ED82AD611
:104280002ED432D236D03ACE3ECC42CA46C872C6BE
:1042900076C47AC27EC0EF00B002F250E2525253AE
:1042A000C2533255A255125682567247E2475248BF
:1042B000C248324EA24E124F824F2161730020300D
:1042C000397106DE16DC1ADA1ED82AD62ED432D27E
:1042D00036D03ACE3ECC42CA46C872C676C47AC2FE
:1042E0007EC0EF00B00AF250E2525253C253325530
:1042F000A255125682567247E2475248C248324E81
:10430000A24E124F824F216173002030397106DEB8
:1043100016DC1ADA1ED82AD62ED432D236D03ACEAD
:104320003ECC42CA46C872C676C47AC27EC0EF008E
:104330009012F250E2525253C2533255A2551256C5
:1043400082567247E2475248C248324EA24E124F3E
:10435000824F216173002030B7070020039787291F
:1043600081472A97634F070009CD05669306F6FF3C
:10437000B6876358C700AA876305D500931707015E
:10438000C1833E858280EFC20F99EFF08FAEEFF0D0
:104390006FBDEFF02FC46FC04F9A3787000003271F
:1043A0008708B707002023A6E72A378700000327DE
:1043B000C708B707002023A4E72A37870000032790
:1043C0000709B707002023A2E72A8280EFC2AF9433
:1043D000B70700200395E729EFF01FF8EF20806F63
:1043E000B707002083A5472AEF2060406FC0EF94F5
:1043F000EFC26F92B70700200395072AEFF0DFF5B1
:10440000EF20406DB707002083A5872AEF20203ECC
:104410006FC0AF92EFC22F90EFF0CFD86FC0EF9187
:10442000EFC26F8F85472E86930500086307F5025C
:104430008947930500106302F5028D47930500201C
:10444000630DF5009147930500406308F50095471B
:10445000631DF500856593850580372501401305AB
:104460000580EFF00FEB6FC04F8D99478565E30630
:10447000F5FE9D478965E302F5FEA1479165E30ED0
:10448000F5FCA547A165E30AF5FCA947E31DF5FC8A
:10449000A145E1B7EFC22F880547930500086308DF
:1044A000E5020947AA87930500106302E5020D475C
:1044B00093050020630DE500114793050040630854
:1044C000E5001547631DE500856593850580372563
:1044D000014013050580EFF08FE46FC00F86194788
:1044E0008565E306E5FE1D478965E302E5FE214794
:1044F0009165E30EE5FC2547A165E30AE5FC294744
:104500001305F00FE39BE7FCA145D1B7EFC2AF80E5
:10451000EFF0AFB16FC06F82EFB2FFFFEFF0EFC10E
:104520006FC0AF81EFB29FFD3704002093070402F4
:104530000149130404021947D4436392A60893095E
:104540004002B3093903330A340183470A0095E76F
:10455000AA841385C9002295EFF08F8B9947032514
:104560008A006390F402EFF06FE193074002330991
:10457000F902854722992300F900330534016FB011
:104580003FFB9D476395F400EFF02FECF9BF89479F
:104590006395F400EFF04FF8C9BFA1476395F400AD
:1045A000EFF01F84D9B78D476395F400EFF01F93A8
:1045B0006DBF9547E39BF4FAEFF03FB47DB7050973
:1045C00093874702E31AE9F6014555BF814709C9B8
:1045D0001821814711C75C49084D898FB337F00016
:1045E0003E858280EFB23FF341112A84A307010088
:1045F000EFF0DFFD19C59305F1001305C400EFF0DE
:10460000EF84888741016FB05FF3EFB2DFF0B70747
:104610000020B765002023A4A7021306001093858D
:10462000C5511945EFF01FF0B707002023A6A72CAE
:104630006FB0BFF0EFB23FEEB7070020B7650020C4
:1046400023A6A704130600109385C5611D45EFF04E
:104650007FEDB707002023A8A72C6FB01FEEEFB2A5
:104660009FEBB7070020B765002023A8A706130615
:1046700000109385C5710945EFF0DFEAB707002008
:1046800023AAA72C6FB07FEBEFB2FFE8B70700209B
:10469000B775002023AAA708130600109385C581CB
:1046A0002145EFF03FE8B707002023ACA72C6FB0FF
:1046B000DFE8EFB25FE6B7070020B775002023AC54
:1046C000A70A130600109385C5910D45EFF09FE5ED
:1046D000B707002023AEA72C6FB03FE6EFB2BFE3D1
:1046E000B7070020B775002023AEA70C13060040C3
:1046F0009385C5A11545EFF0FFE2B707002023A081
:10470000A72E6FB09FE3B707002083A7C72C63993C
:10471000A700B707002083C7472E858B3E85828080
:10472000B707002083A7072D6398A700B7070020CD
:1047300083C7472E898BDDB7B707002083A7472D96
:104740006398A700B707002083C7472E918BF9B75E
:10475000B707002083A7872D6398A700B70700201D
:1047600083C7472EA18B5DBFB707002083A7C72D46
:104770006399A700B707002083C7472E93F7070266
:1047800071BFB707002003A7072E9307F00FE317A9
:10479000E5F8B707002083C7472E93F70704BDBF8E
:1047A0008547631BF500B70700209387472E9823A2
:1047B0001367170098A382807DFDB70700209387B9
:1047C000472E9823799BFDB78547631BF500B707F4
:1047D00000209387472E98231367270098A3828091
:1047E0007DFDB70700209387472E9823759BFDB763
:1047F0008547631BF500B70700209387472E982352
:104800001367470098A382807DFDB7070020938738
:10481000472E98236D9BFDB78547631BF500B707AF
:1048200000209387472E98231367870098A38280E0
:104830007DFDB70700209387472E98235D9BFDB72A
:104840008547631BF500B70700209387472E982301
:104850001367070298A382807DFDB7070020938726
:10486000472E98231377F7FDF5B78547631BF500AF
:10487000B70700209387472E98231367070498A350
:1048800082807DFDB70700209387472E98231377FA
:10489000F7FBF5B7EFB23FC83745004093055052DC
:1048A00013050540EFC01F9F31C5B7070020938750
:1048B000972B982309E7054798A3EF003010374559
:1048C000004013050540EFC0DF9B9375F50FB70758
:1048D0000020238EB72AB707002003A5472D1C4DC3
:1048E000104954498507B3E7C7026385D7003105EE
:1048F000EFE01FD337440040930570721305044066
:10490000EFC05F991DCDB707002083A7472D9633D1
:10491000BA3363EDE6000146930570721305044057
:10492000EFC05F92EF10204F6FB03FC1D84F13869A
:10493000160092B3B307D7008C2313050440EFC0D1
:10494000DF93374400409305404213050440EFC015
:104950007F9479D90357044083574440EF00207C6B
:10496000E1B7EFB25FBB37550040930550521305D6
:104970000580EFC03F9231C5B70700209387172C01
:10498000982309E7054798A3EF00D0063755004064
:1049900013050580EFC0FF8E9375F50FB707002054
:1049A0002382B72CB707002003A5C72D1C4D104943
:1049B00054498507B3E7C7026385D7003105EFE0A7
:1049C0003FC6375400409305707213050480EFC052
:1049D0007F8C1DCDB707002083A7C72D9633BA3330
:1049E00063EDE60001469305707213050480EFC085
:1049F0007F85EF1080446FB05FB4D84F13861600E8
:104A000092B3B307D7008C2313050480EFC0FF8651
:104A1000375400409305404213050480EFC09F8740
:104A200079D90357048083574480EF008073E1B73E
:104A3000EFB27FAE9305505237550040EFC09F85CF
:104A400015C937550040EFC0DF839375F50FB707E1
:104A500000202384B72CB707002003A5072E1C4D88
:104A6000104954498507B3E7C7026385D70031056C
:104A7000EFE01FBB9305707237550040EFC09F8178
:104A800015C1B707002083A7072E9633BA3363ED0D
:104A9000E60001469305707237550040EFC08FFA6B
:104AA000EF10C03A6FB07FA9D84F1386160092B3AB
:104AB000B307D7008C2337550040EFC00FFCDDB79C
:104AC000EFB27FA5372500409305505213050580AE
:104AD000EFC04FFC31C5B70700209387072B982301
:104AE00009E7054798A3EF00E06937250040130563
:104AF0000580EFC00FF99375F50FB7070020238AE3
:104B0000B72AB707002003A5C72C1C4D10495449EC
:104B10008507B3E7C7026385D7003105EFE05FB0D3
:104B2000372400409305707213050480EFC08FF6A0
:104B30001DCDB707002083A7C72C9633BA3363ED8A
:104B4000E60001469305707213050480EFC08FEFF5
:104B5000EF10202A6FB07F9ED84F1386160092B3B5
:104B6000B307D7008C2313050480EFC00FF137245F
:104B700000409305404213050480EFC0AFF179D99E
:104B80000357048083574480892BE9B7EFB2BF985D
:104B90003725004093055052130505C0EFC08FEF35
:104BA00029C5B70700209387572B982301E70547AE
:104BB00098A3FD2337250040130505C0EFC06FEC17
:104BC0009375F50FB7070020238CB72AB70700208D
:104BD00003A5072D1C4D104954498507B3E7C702AB
:104BE0006385D7003105EFE0BFA33724004093056C
:104BF0007072130504C0EFC0EFE91DCDB7070020A8
:104C000083A7072D9633BA3363EDE600014693057B
:104C10007072130504C0EFC0EFE2EF10A01E6FB07A
:104C2000DF91D84F1386160092B3B307D7008C23B9
:104C3000130504C0EFC06FE43724004093054042E1
:104C4000130504C0EFC00FE579D9035704C083579B
:104C500044C06D21E9B7EFB21F8C93055052372540
:104C60000040EFC02FE339C1B70700209387D72B4F
:104C7000982301E7054798A3852337250040EFC017
:104C80004FE09375F50FB70700202380B72CB707C7
:104C9000002003A5872D1C4D104954498507B3E713
:104CA000C7026385D7003105EFE09F9793057072C7
:104CB00037250040EFC00FDE1DCDB707002083A7CA
:104CC000872D9633BA3363EDE60001469305707283
:104CD00037250040EFC00FD7EF1000156FB0FF85EC
:104CE000D84F1386160092B3B307D7008C2337250D
:104CF0000040EFC08FD89305404237250040EFC0F9
:104D00006FD969DDB72700409A23DE231529F9B74B
:104D1000EFB27F8041112A842EC632C4EFF0BF9ECD
:104D20002A8955E1B2452246B707002083A4C72C43
:104D30004CCC2310040232B0639184040545EFF09B
:104D40003FA637250140054693050002130505805F
:104D5000EFC00F9805469305707237240040130585
:104D60000480EFC02FCE9A30DC4C130504809306EC
:104D7000170096B0BA978C23A9A0B707002083A488
:104D8000072D639684040545EFF01FA437250140E5
:104D900005469305000413050580EFC06F93372483
:104DA000004093057072130504C00546EFC08FC91B
:104DB0009A30DC4C130504C09306170096B0BA97DE
:104DC0008C23EFC08FCB4A8541016FB00FF7B70737
:104DD000002083A4472D639084040545EFF05FA174
:104DE000371501400546894513050580EFC04F8EF4
:104DF0003744004093057072130504400546EFC028
:104E00006FC49A30DC4C130504409306170096B02B
:104E1000BA978C237DB7B707002083A4872D639EA4
:104E200084020545EFF05F9F371501400546854533
:104E3000130505C0EFC0CF89930570723725004078
:104E40000546EFC02FC09A30DC4C37250040930652
:104E5000170096B0BA978C23ADB7B707002083A48C
:104E6000C72D639484020545EFF09F9D37150140DF
:104E700005469305001013050540EFC06F850546F4
:104E80009305707237540040D9BDB707002083A442
:104E9000072EE39A84F20545EFF03F9D930570726B
:104EA000375500400546EFC0EFB99A30DC4C375516
:104EB00000409306170096B0BA978C2319B7B7072E
:104EC000002083A7C72C6399A700B707002083C7DA
:104ED000072B858B3E858280B707002083A7072D8F
:104EE0006397A700B707002083C7572BDDB7B70725
:104EF000002083A7472D6397A700B707002083C72B
:104F0000972BC1BFB707002083A7872D6397A70002
:104F1000B707002083C7D72B6DBFB707002003A7B3
:104F2000C72D9307F00FE317A7FAB707002083C731
:104F3000172C45B78280EFB20FDE09E9B7070020D2
:104F4000A384072CEFE01FF66FB02FDF954763199E
:104F5000F500B7070020A384A72CEFF08F88EDB7EA
:104F600099476319F500B7070020A384A72CEFF039
:104F7000CF8AD9BF9D476319F500B7070020A384E6
:104F8000A72CEFF00F8DC9B7A1476319F500B7073C
:104F90000020A384A72CEFF04F8F7DB7A547E31522
:104FA000F5FAB7070020A384A72CEFF08F9169BF13
:104FB000B707002003C5972C8280EFB2CFD5B70783
:104FC000002003A5C72D8145EFF0DFF66FB0EFD6C7
:104FD000EFB26FD4B707002003A5872D8145EFF00E
:104FE0007FF56FB08FD5EFB20FD3B707002003A5C1
:104FF000472D8145EFF01FF46FB02FD4EFB2AFD142
:10500000B707002003A5072D8145EFF0BFF26FB071
:10501000CFD2EFB24FD0B707002003A5C72C8145F0
:10502000EFF05FF16FB06FD1EFB2EFCE3757000006
:10503000378500001307270185460146BD45130546
:105040004509EFE00FBAB707002023A4A72E375772
:105050000000378500001307C7FF89460146BD459C
:105060001305C509EFE0EFB7B707002023A6A72E69
:105070003757000037850000130767FE8D4601464D
:10508000BD451305450AEFE0CFB5B707002023A8BB
:10509000A72E3757000037850000130707FD9146FC
:1050A0000146BD451305C50AEFE0AFB3B7070020C1
:1050B00023AAA72E37570000378500001307A7FB48
:1050C00095460146BD451305450BEFE08FB1B70787
:1050D000002023ACA72E6FB04FC6EFB2CFC3B707E7
:1050E000002003A4872EEFD04FDB2A86014781469C
:1050F00099452285EFE02FB66FB02FC4EFB2AFC154
:10510000B707002003A4C72EEFD02FD92A86014766
:10511000814699452285EFE00FB46FB00FC2EFB220
:105120008FBFB707002003A4072FEFD00FD72A8621
:105130000147814699452285EFE0EFB16FB0EFBF9F
:10514000EFB26FBDB707002003A4472FEFD0EFD415
:105150002A860147814699452285EFE0CFAF6FB09F
:10516000CFBDEFB24FBBB707002003A4872FEFD00E
:10517000CFD22A860147814699452285EFE0AFAD1F
:105180006FB0AFBBEFB22FB9B707002003A5872ED2
:10519000014781460146A145EFE0EFAB6FB0EFB9A3
:1051A000EFB26FB7B707002003A5C72E01478146AE
:1051B0000146A145EFE02FAA6FB02FB8EFB2AFB50F
:1051C000B707002003A5072F014781460146A145E7
:1051D000EFE06FA86FB06FB6EFB2EFB3B707002084
:1051E00003A5472F014781460146A145EFE0AFA641
:1051F0006FB0AFB4EFB22FB2B707002003A5872F6F
:10520000014781460146A145EFE0EFA46FB0EFB240
:10521000EFB26FB02A84EFF00FCF01E92285EFF0F3
:105220001FCA3335A0006FB04FB10545EDBFEFB2D7
:105230008FAEEFF04FCD6FB04FB0EFB24FABB704C2
:10524000002083D7C42F41119384C42F89E7EFD066
:105250002FC423A4A190EFD0AFC337790020AA8A2E
:10526000094BB7090020854B130A30061309C9E121
:105270005685EF10804D6360AB0A03A5C92CEFF093
:10528000EFB4631A75098220637D8A068220EFC01D
:10529000EFAB9307E4406363F5061305E400EFC04A
:1052A000EF8792202AC61304D500930766001CC11D
:1052B000930785005CC1930730051CA59307C004C4
:1052C0001CB585473CA5B7750020935786003CB5B3
:1052D00050A59385C5E12285EF1030308A20DD4747
:1052E00022951CA103A58196EFC05FE829C503A5FF
:1052F0008196814629466C00EFC02FF6239004006A
:1053000005A803A5C92C930714009EA04A94EFF0AA
:105310006FAD08A0B1BF9A2093073006E3E8E7F627
:1053200003A58190EF10604293072003E3E0A7F606
:1053300041016FB04F9F3245EFC0EF96C1B7EFB25A
:105340000F9BB704002083D7E42F41119384E42FEF
:1053500089E7EFD0EFB323A6A190EFD06FB33779F1
:105360000020AA8A094BB7090020854B130A300692
:105370001309C9E95685EF10403D6360AB0A03A5E8
:10538000092DEFF0AFA4631A75098220637D8A06A8
:105390008220EFC0AF9B9307E4406363F5061305DB
:1053A000E400EFB0BFF792202AC61304D50093079C
:1053B00066001CC1930785005CC1930730051CA5DE
:1053C0009307C0041CB589473CA5B77500209357C7
:1053D00086003CB550A59385C5E92285EF10F01FE6
:1053E0008A20DD4722951CA103A58196EFC01FD816
:1053F00029C503A58196814629466C00EFC0EFE5DB
:105400002390040005A803A5092D930714009EA06E
:105410004A94EFF02F9D08A0B1BF9A209307300661
:10542000E3E8E7F603A5C190EF10203293072003CD
:10543000E3E0A7F641016FB00F8F3245EFC0AF86B2
:10544000C1B7EFB2CF8A83D7019041119384019005
:1054500089E7EFD0EFA323A8A190EFD06FA337790E
:105460000020AA8A094BB7090020854B130A300691
:105470001309C9F15685EF10402D6360AB0A03A5EF
:10548000492DEFF0AF94631A75098220637D8A0677
:105490008220EFC0AF8B9307E4406363F5061305EA
:1054A000E400EFB0BFE792202AC61304D5009307AB
:1054B00066001CC1930785005CC1930730051CA5DD
:1054C0009307C0041CB58D473CA5B77500209357C2
:1054D00086003CB550A59385C5F12285EF10F00FED
:1054E0008A20DD4722951CA103A58196EFC01FC825
:1054F00029C503A58196814629466C00EFC0EFD5EA
:105500002390040005A803A5492D930714009EA02D
:105510004A94EFF02F8D08A0B1BF9A209307300670
:10552000E3E8E7F603A50191EF102022930720039B
:10553000E3E0A7F641016FA01FFF3245EFB0BFF6D1
:10554000C1B7EFA2DFFA83D7219041119384219054
:1055500089E7EFD0EF9323AAA190EFD06F9337792B
:105560000020AA8A094BB7090020854B130A300690
:105570001309C9F95685EF10401D6360AB0A03A5F6
:10558000892DEFF0AF84631A75098220637D8A0646
:105590008220EFB0BFFB9307E4406363F506130579
:1055A000E400EFB0BFD792202AC61304D5009307BA
:1055B00066001CC1930785005CC1930730051CA5DC
:1055C0009307C0041CB591473CA5B77500209357BD
:1055D00086003CB550A59385C5F92285EF10E07F84
:1055E0008A20DD4722951CA103A58196EFC01FB834
:1055F00029C503A58196814629466C00EFC0EFC5F9
:105600002390040005A803A5892D930714009EA0EC
:105610004A94EFE03FFD08A0B1BF9A2093073006FF
:10562000E3E8E7F603A54191EF102012930720036A
:10563000E3E0A7F641016FA01FEF3245EFB0BFE6F0
:10564000C1B7EFA2DFEA83D7419041119384419023
:1056500089E7EFD0EF8323ACA190EFD06F83377948
:105660000020AA8A094BB7090020854B130A30068F
:105670001309C9015685EF10400D6361AB0A03A5FC
:10568000C92DEFE0BFF4631B75098220637E8A0693
:105690008220EFB0BFEB9307E4406364F506130587
:1056A000E400EFB0BFC79E202AC62A8499071CC118
:1056B000930785005CC1930730051CA59307C004C0
:1056C0001CB5EFF0FF8E922028A4B77500209357E9
:1056D00086003CB450A4350422859385C501EF10A3
:1056E000C06F9E203E94DD471CA003A58196EFC0AD
:1056F000FFA729C503A58196814629466C00EFC006
:10570000CFB52390040005A803A5C92D9307140065
:105710009EA04A94EFE01FED08A0A9BF9A2093072E
:105720003006E3E7E7F603A58191EF100002930747
:105730002003E3EFA7F441016FA0FFDE3245EFB095
:105740009FD6C1B7EFA23FDDAD23FDBFEFA2BFDC07
:10575000EFF0BFAEEFF0BFBEEFF0BFCEEFF07FDEF9
:10576000EFF03FEE1545EFD00FB2DDB7EFA2BFDA95
:10577000370400200325042EEF00307E5145EFD082
:105780008FB0CDBFEFA23FD9C12CFDBFEFA2BFD8D4
:105790004111EFC0FFEF2AC60144E54437890000FC
:1057A000EFE0DFC2612AEFE0BFC45D22631D940019
:1057B000EFB0DFD9AA861306A00685451305090CAC
:1057C000EF10A04F01440504420493054006680011
:1057D0004180EFD04F9EE9B7EFA2FFD3EFE01FD398
:1057E000DD28EFE03FC3EFE01FBAEFE01FBB9D2ACB
:1057F000EFE0DFEEAD2AEFE05FE1BD2AEFE09FE3EF
:105800004922EFE0DFE55922EFE01FE86922EFE0EF
:105810005FEA7922DD26EFF03F811305803EEFD06D
:105820005FCEEFE08FB085452945EFE07FBFB785BC
:105830000000375500009387C19109478146130640
:1058400000209385C50E1305C578EFC03FBAB78514
:10585000000037550000938781921D47814613064B
:1058600000109385850F13054578EFC03FB8B785C5
:105870000000375500009387C192154781461306F3
:105880000010938585101305C576EFC03FB6B78528
:105890000000375500009387019211478146130697
:1058A0000040938585111305C574EFC03FB4B785DB
:1058B0000000375500009387419215478146130633
:1058C00000109385851213054574EFC03FB2EFC0F9
:1058D0003FD26FA09FC6EFA21FC401116946814548
:1058E0004800EFE07FC3E145A0864800EF00206F4D
:1058F000B77700209387C7096311A402224798CB8A
:105900003247D8CB424798CF5247D8CF624798D337
:105910001247D8C705616FA05FC209671307075810
:1059200098CBD8CB98CFD8CF71671307072098D3DF
:10593000CDB7B777002003A5C7098280B7770020CD
:1059400023AEA7088280B777002003A5070A8280CC
:10595000B777002023A0A70A8280B777002003A58D
:10596000470A8280B777002003A5870A8280B7772D
:10597000002003A5C70A8280B777002003A5070B84
:105980008280B777002003A5470B8280B77700207D
:1059900003A5870B8280B777002003A5C70B828001
:1059A000EFA2DFB5014691451545EFC00F84138B7B
:1059B00041932320AB00014691451545EFC0EF828E
:1059C000938AC19323A0AA00014691451545EFC0D3
:1059D000CF81138A41942320AA00014691451545A1
:1059E000EFC0AF809389C19423A0A90001469145DF
:1059F0002945EFB09FFF1389419501462320A90057
:105A000091452945EFB07FFE9384819688C0194562
:105A100013840196EFC07F86AA8508C003250B007A
:105A2000EFC0BF860C4003A50A00EFC01F860C40E4
:105A300003250A00EFC07F850C4003A50900EFC0D5
:105A4000DF840C4003250900EFC03F840C408840F0
:105A5000EFC0BF836FA0DFADEFA25FAA03A50196E1
:105A6000FD55B7090020EFC03F8523A6A19603A5E9
:105A7000092E1384C195EFF08FFB0DE903A58196E4
:105A8000B77400209384040C014693850401EFC091
:105A9000CFBB85472A89631BF5009C4803A5092EC7
:105AA0009223CC43EFF0CFA6230024013709002036
:105AB0000325C92CEFF0CFF50DE903A54193B77588
:105AC00000209389050C01469385050CEFC0EFB7C4
:105AD0008547AA84631BF50083A709000325C92C09
:105AE0009223CC43EFF0CFA204A0B709002003A576
:105AF000092DEFF0EFF10DE903A5C193B774002074
:105B00009384040C014693854400EFC00FB485478D
:105B10002A89631BF500DC4003A5092D9223CC43A1
:105B2000EFF00F9F23002401B709002003A5492DA2
:105B3000EFF00FEE0DE903A54194B77400209384B4
:105B4000040C014693858400EFC02FB085472A8955
:105B5000631BF5009C4403A5492D9223CC43EFF031
:105B60002F9B23002401B709002003A5892DEFF006
:105B70002FEA15E903A5C194B77400209384040C9F
:105B800001469385C400EFC04FAC85472A89631C4A
:105B9000F500D8449C4403A5892D1223CC43EFF093
:105BA0002F9723002401370900200325C92DEFF08A
:105BB0002FE615ED03A54195B77400209384040CDE
:105BC000014693854401EFC04FA885476311F50254
:105BD000DC488823EFF02FB6DC480325C92DD223FB
:105BE0008C47EFF0EF92230004006FA07F941C20FD
:105BF000FDFB0D45EFC03FE9FDB7EFA23F90194512
:105C000013840193EFC06FE708C00D468145054539
:105C1000EFB0BFDD138B81932320AB000D46814590
:105C20000545EFB09FDC938A019423A0AA000D469E
:105C300081450545EFB07FDB138A81942320AA00BC
:105C40000D4681450545EFB05FDA9389019523A0A4
:105C5000A9000D4681450545EFB03FD913898195CF
:105C60000D462320A90081450545EFB01FD8938438
:105C7000419688C00C4003250B00EFC00FE10C409B
:105C800003A50A00EFC06FE00C4003250A00EFC037
:105C9000CFDF0C4003A50900EFC02FDF0C40032528
:105CA0000900EFC08FDE0C408840EFC00FDE6FA010
:105CB0003F88EFA25F8603A50193FD55EFC0CFDFBC
:105CC000138481931C40639DA702B777002003A52E
:105CD000070CEFB04FFD0545EFC0FFDA3725014057
:105CE00013050580014693050002EFB06F9E014544
:105CF000EFE01FAB08408145EFC08FAB6FA0FF8383
:105D0000138401941C406398A702B777002003A571
:105D1000470CEFB04FF90545EFC0FFD637250140DE
:105D200001469305000413050580EFB06F9A014505
:105D3000EFE09FA9C1B7138481941C406397A70229
:105D4000B777002003A5870CEFB0EFF50545EFC04E
:105D50009FD3371501400146894513050580EFB0F3
:105D60002F970145EFE0DFA871B7138401951C4020
:105D70006397A702B777002003A5C70CEFB0AFF277
:105D80000545EFC05FD03715014001468545130535
:105D900005C0EFB0EF930145EFE01FA8A1BF13844A
:105DA00081951C406398A702B777002003A5470D93
:105DB000EFB06FEF0545EFC01FCD3715014001462D
:105DC0009305001013050540EFB08F900145EFE0FB
:105DD0003FA70DB7138441961C40E391A7F2B77714
:105DE000002003A5070DEFB00FEC0145EFE0FFA782
:105DF00011B7EFA24FF203A581938145EFB0FFF3F6
:105E00006FA0AFF3EFA22FF103A501948145EFB08E
:105E1000DFF26FA08FF2EFA20FF003A5819481450E
:105E2000EFB0BFF16FA06FF1EFA2EFEE03A5019508
:105E30008145EFB09FF06FA04FF0EFA2CFED03A52B
:105E400081958145EFB07FEF6FA02FEFEFA2AFEC10
:105E500003A541968145EFB05FEE6FA00FEEEFA274
:105E60008FEB2545EFE00FE36FA02FEDEFA2AFEA38
:105E70002145EFE02FE26FA04FECEFA2CFE91D45E7
:105E8000EFE04FE16FA06FEBEFA2EFE81945EFE015
:105E90006FE06FA08FEAEFA20FE81545EFE08FDF0C
:105EA0006FA0AFE9EFA22FE71145EFE0AFDE6FA0E3
:105EB000CFE8EFA24FE60D45EFE0CFDD6FA0EFE7B3
:105EC000EFA26FE50945EFE0EFDC6FA00FE7EFA26F
:105ED0008FE40545EFE00FDC6FA02FE6EFA2AFE304
:105EE000EFF0BFA7B787000083A58713EF0030103E
:105EF000EF00F038420541816FA02FE4EFA2AFE13F
:105F0000EFF07FA4B787000083A58713EF00300E62
:105F1000EF00F036420541816FA02FE2EFA2AFDF24
:105F2000EFF03FA1B787000083A58713EF00300C87
:105F3000EF00F034420541816FA02FE0EFA2AFDD0A
:105F40000C212545EFE0CFCD01456FA00FDFEFA27B
:105F50008FDC0C212145EFE0AFCC01456FA0EFDDD8
:105F6000EFA26FDB0C211D45EFE08FCB01456FA049
:105F7000CFDCEFA24FDA0C211945EFE06FCA0145E3
:105F80006FA0AFDBEFA22FD90C211545EFE04FC971
:105F900001456FA08FDAEFA20FD80C211145EFE079
:105FA0002FC801456FA06FD9EFA2EFD60C210D4588
:105FB000EFE00FC701456FA04FD8EFA2CFD50C215E
:105FC0000945EFE0EFC501456FA02FD7EFA2AFD491
:105FD0000C210545EFE0CFC401456FA00FD6C16786
:105FE00069768146FD1705061397060141836364B0
:105FF000B7003E8582803307D5001823B98F21472B
:1060000013F81700858363050800B18FC207C183A9
:106010007D17420741836DF78506F9B7EFA20FCED2
:106020001389219783D401970354090081499387E9
:10603000F4FF634CF4029385D4FF377A0020930A6F
:106040008A0D93F5F50F13058A0DEFF05FF9D694DD
:1060500083C7D4FF03C7E4FFA207D98F13878197B3
:106060006318F50095471CC385494E856FA04FCC3A
:106070001306F4FF4206418293851A0013058A0D28
:10608000232007002310C900EF001038F9BFEFA24A
:106090000FC6938481979C403971B1EF03D6219745
:1060A00085469387219763F9C60237750020130749
:1060B000850D03480700930830059305850D63108F
:1060C000180314331307C004639BE652B1479CC006
:1060D000EFC00FDC23AAA19621616FA0CFC4930863
:1060E0007004631E185103481700130770056318E6
:1060F000E85094C0F1BF0547138481976397E70484
:10610000377700200347A70DC1461376F70D6308C4
:10611000D600130707031377F70F63E5E7008947F6
:106120001CC05DBF938721979223232004007D1616
:106130004206418292A3377500209305850D85059F
:106140001305850DEF00502C41BF09476393E70A03
:1061500003D62197114793862197E37FC7F63775BA
:1061600000209307850DB823130800039305850DC0
:10617000631F0701B833DC232207D98F25476364E7
:10618000F74429472398E1968D479CC0B1B7414811
:10619000631B0701B833DC232207D98F25476364CB
:1061A000F7429D47DDB71308000D63180701B833A8
:1061B000DC2363EAE740A547C9BF1308100D631449
:1061C0000741D82303C83700220733670701931715
:1061D00087002183D98FC207C1831388F7FF130774
:1061E000E0046362073F2D4798C0A1072398F1960A
:1061F000E5B50D476390E70403D6219799461387C9
:10620000219763FFC600B77600209386860DDC32A7
:10621000F422A207D58FCD4663E7F6009147B5B7C4
:106220009147E3FBC7EA7D16420641822320040022
:1062300012A311B71147639FE7049389219703D4F1
:106240000900A147E3FA87E803D90197377A0020CC
:10625000930A8A0D9305D9FF93F5F50F13058A0D5F
:10626000EFF0FFD756998347D9FF0347E9FFA2070D
:10627000D98F6394A700954709BF1306F4FF420620
:10628000418223A004002390C90093851A001305BE
:106290008A0D4DBD15476397E70203D6219703D7B3
:1062A000019737750020938721979305850D631615
:1062B000E6343387C5008346F7FF5947639FE632CC
:1062C000BD47B9BD99466390D720B7740020938726
:1062D000840DB823930700039384840D631CF70C8B
:1062E00083C93400DC2003C95400A209B3E9F900D2
:1062F000FC202209130680023369F9004209135970
:106300000941931B09018145280893DB0B01EFA08C
:106310008FA3130A81014E8B370C0020B3073B413A
:10632000C207C18363E3770F910B93991B00EFB012
:10633000EFA193878940636FF50613858900EFA06D
:10634000FFFD930785005CC1930770042ACA1CA552
:1063500093077005232035011CB5E119930700034D
:106360003CA5060993D789403CB5230625011307B0
:10637000D500814763CF370B484193951B00F51536
:1063800093F5F50FBA99EFF09FC5935785002380D9
:10639000F900D947A380A9002381F90003A58196BC
:1063A000EFB0DFDC45C903A58196814629464C083C
:1063B000EFB0AFEAB820C147631CF70C03CA340042
:1063C000DC2083C95400220A336AFA00FC20A209A7
:1063D0001306800281452808B3E9F90013098101F9
:1063E000EFA06F96CA86814789046399F906D28A1D
:1063F000370B0020B3874A41C207C18363EA3707DE
:106400002320040023990196C1B9930A8C0F938C21
:106410000A0683A70A006398670183A74A0001451B
:1064200082972310AA00A10AE3959AFF090A050B97
:10643000F5B58C0093F6E70FAE9693F5170033068B
:10644000F70083D686FD91E1A182850714A293F718
:10645000F70F0DB75245EFB00F85A9BFD824D03440
:1064600085072207518FC2079AA2C1838906ADBF53
:1064700093048B15938B84049C4063955701DC40F7
:106480004A858297A104E39974FF0909850A9DB79B
:106490009C341307000D639CE7003785000013064A
:1064A000D04585451305C513EF00300191BF130793
:1064B000100DE397E7F43785000013067046854515
:1064C00013058517D5B71D47639BE70203D62197B0
:1064D00013872197E3F2C6C0377500209306850D18
:1064E000DC32F4229305850DA207D58FCD4663ECEF
:1064F000F604950786072398F196914715B1214731
:106500006395E700EFF09FB1C1BE25476394E704B0
:106510001387219712239947E3F0C7BC37750020F2
:106520009305850DD62593978600A182D58FC20746
:10653000C1831388F7FF9306500E63E606012947CF
:1065400018C0A90765B17D164206418223200400C8
:1065500012A3F5B629476395E700EFF03FACADBE57
:106560002D476395E700EFF07FABBDB63147639BE6
:10657000E700B777002003C7A70DA547E3E4E7BA14
:10658000B54779BE35476397E704938621979222F2
:106590009147E3F3C7B4377500209305850DD821E3
:1065A000BC3122075D8F931787002183D98FC207E3
:1065B000C1831388F7FF1307F03F6366070139476C
:1065C00018C0990725B17D16420641822320040098
:1065D00092A2B5B639476399E70293872197922330
:1065E00003D70197E36AE6AE377500209305850D62
:1065F0002E978346F7FF5D47D1B1232004007D1617
:106600004206418292A325BE3D47E397E7AC377926
:1066100000201307890D5C2324331309890DA20779
:10662000C58F93948700A183DD8CC204C180EFA045
:10663000FFF193870440E365F5DC83472900138667
:1066400014000D47FD1793F7F70F32C6B7790020F6
:106650006362F70413858400EFA05FCC32462ACC36
:10666000AA8710C12105C8C39385D90DEF00E07634
:10667000834729000547639AE70203A54193EFB0DA
:10668000FFAE61C103A54193814629462C08EFB0B6
:10669000CFBCBDB31385C400EFA05FC832462ACC7F
:1066A000AA8750C1310588C7C1B70947639DE70074
:1066B00003A5C193EFB09FAB49C5814629462C087D
:1066C00003A5C193E9B70D47639DE70003A5419476
:1066D000EFB0DFA93DC5814629462C0803A54194AA
:1066E0007DB71147639DE70003A5C194EFB01FA8D4
:1066F00029C9814629462C0803A5C19449BF1547DD
:10670000639FE70062471CA303A54195EFB01FA656
:106710000DC9814629462C0803A541958DBF19470F
:10672000E382E7FE1D47E38FE7FC2147E38CE7FCAC
:106730002547E389E7FCE39507CCE2472380070080
:10674000E1B76245EFA03FD665B9EF92DFDC2A845E
:10675000EFB01FF4018D6F905FDEEF923FDA13848C
:106760004197AA84EFB0DFF20329040023AEA1967B
:10677000EFB01FF2330525419307703E9389C1970F
:1067800063F9A700EFB0DFF02399019608C023ACAE
:10679000019637790020854A114A1309890D26850B
:1067A000EFD0DFE2630A55012685EFD03FE285474F
:1067B0006319F5026F90DFD7EFB09FED83A7090053
:1067C0001D8DE363AAFE93872197822326851307F5
:1067D00014009AA34A94EFD0FFE008A0EFF03F8B9B
:1067E0007DBF83A78197F9D7EFF07F8AE1B77971F1
:1067F00022D4135475014ECE52CC9319950006D66F
:1068000026D24AD056CA5AC81374F40F93D99900A5
:10681000135AF50169C49307F00F6308F40E9397B8
:10682000390037070004B3E9E700130414F8814482
:10683000014B13D77501939A95001377F70F93DAED
:106840009A0013D9F50145CF9307F00F630CF702B7
:106850008E0A130717F8B7070004B3EAFA003A9450
:10686000014633452A01BD47AA869305140063E01B
:106870009710172700001307A7938A04BA949C4027
:10688000BA9782871304F40F63960A0C93E42400EA
:106890000946C1BF01451307F00FB7074000B250CA
:1068A0002254A6075E07A5837E05D98F925402590C
:1068B000F249624AD24A424B5D8D45618280CA8666
:1068C000D689328B8947630FFB088D47E304FBFCB5
:1068D000854736856310FB1A01478147C9B7639D19
:1068E000090413D77501939A95001377F70F914414
:1068F0000144054B93DA9A0013D9F50131F7639DF2
:106900000A0093E414000546A9BF63920902A1445A
:106910001304F00F094B31BF568541249307B5FF8F
:10692000098CB39AFA001304A4F801461DBFB144C0
:106930001304F00F0D4BF5BD4E852EC6B92C9307F1
:10694000B5FF1304A0F8B399F900098C8144014BF9
:10695000B245C5B593E434000D4621B78947D286C8
:10696000E315FBF636851307F00F81470DBF416332
:106970009306F3FF13D6090193D80A01B3F7D900A0
:10698000B3FADA0033885703B389F80213570801C2
:10699000B30A5603D6994E9733061603637357010D
:1069A0001A96C167FD17B376F7003378F800C20670
:1069B000C2969399660093570701B3393001E98273
:1069C000B2979A07B3E6D900B3E9D7009397490085
:1069D00063D9070013D7190093F71900B369F700BB
:1069E0002E841307F4076350E00493F7790099C7E6
:1069F00093F7F90091466383D70091099397490073
:106A000063D90700B70700F8FD17B3F9F9001307BA
:106A100004089307E00F63CBE70493976900A5830D
:106A20001377F70FADBD8547B386E74011C76D46B5
:106A300001478147E345D6E61307E4093397E900A8
:106A40003337E000B3D7D900D98F13F7770019C7D0
:106A500013F7F70091466303D70091071397570088
:106A6000634C07009A07A583014715BD1307F00F74
:106A7000814735B52E84B5B7054781470DB5135706
:106A80007501370680009307F6FF1377F70F93051C
:106A9000E007B3F6A7009357F501014563F4E5005D
:106AA00099C3828082809307E0097D55E3EBE7FE7E
:106AB00093055009B3E7C60063D7E5001307A7F6AF
:106AC0003395E7008280130560093307E54033D52D
:106AD000E7008280411106C622C426C20DCD93571D
:106AE000F54133C4A7001D8CAA8422857D2093071D
:106AF000E0093387A74093076009FD8063CCE70274
:106B0000A1469377F70F63D5A60061153314A4004F
:106B10002604258021A08144814701442604135581
:106B20009400B2402244DE07FE045D8D458D924400
:106B3000410182809307900963DDE7009307B50167
:106B40009546B317F400898E3354D400B337F00060
:106B50005D8C954763D6A7009307B5FF3314F40007
:106B6000B70600FCFD16937774003376D40085C316
:106B70009377F4009145638CB70011069317560084
:106B800063D707009307F009758E3387A740131466
:106B9000660025809377F70F51B7C167637CF502D4
:106BA0009307F00F1307000263EBA700971700008D
:106BB00093870764AA9788233305A74082802181A1
:106BC000971700009387C762AA9788236147330508
:106BD000A7408280B7070001636DF50061819717B8
:106BE00000009387E760AA97882321473305A740D1
:106BF00082804181971700009387875FAA97882337
:106C000041473305A7408280B3C7A5008D8B33076A
:106C1000C50081E78D4763EDC700AA87637EE5085D
:106C2000942185078505A38FD7FEE3EBE7FE8280DD
:106C300093763500AA8789CA942185078505A38F95
:106C4000D7FE93F63700C5BF9376C7FF138606FEBF
:106C500063F0C70683A3050083A2450083AF8500C8
:106C600003AFC50083AE050103AE450103A3850153
:106C700083A8C5019385450223A0770003A8C5FF1B
:106C800023A2570023A4F70123A6E70123A8D701D5
:106C900023AAC70123AC670023AE170193874702DD
:106CA00023AE07FF75B790419107910523AEC7FE4C
:106CB000E3EBD7FEE3E6E7F6828039713EDA2ED2C7
:106CC00032D436D63AD842DC46DE9387418122CC94
:106CD000804326CA06CEAA8409C41C4C99E32285A7
:106CE000352B0C4454102686228536C6EF007017CB
:106CF000F2406244D24421618280011126CA4AC80E
:106D000006CE22CC4EC652C4AA842E8901C51C4D83
:106D100091E329239C4C804499E32685012397170E
:106D200000009387E75E631BF402C0405E24A18BE2
:106D3000B1C71C48A1C7FD59294A1C448345090015
:106D4000FD17B1E91CC463DD07062286A945268527
:106D5000E120FD576308F502294535A0971700008B
:106D60009387075D6314F4008044C9B79717000048
:106D700093870758E31CF4FAC0444DBFA2852685CB
:106D8000912A55D97D55F2406244D2444249B249D4
:106D9000224A056182801CC4050963D70700184C8C
:106DA00063CAE700638845011C401387170018C0B9
:106DB0008CA361B7228626858520E31035F9D9B7E3
:106DC0001C401387170018C0294798A371B79387F1
:106DD0004181AA8588436FF05FF205C68547630B42
:106DE000F602138715002E968346F7FF0505BA872E
:106DF000A30FD5FE81CE0507E318E6FE23000500AC
:106E000011A0AE87850703C7F7FF6DFF3385B74035
:106E10007D158280AE87DDB7011122CC26CA4AC813
:106E200006CE4EC6AA842E89328401C51C4D91E33C
:106E3000F526971700009387A74D6317F406C04007
:106E40001C4C1CC45E24A18BC1C31C48B5CF1C487C
:106E500008409379F90F1379F90F1D8D5C4863464B
:106E6000F500A2852685692C25E51C440505FD173E
:106E70001CC41C401387170018C0238037015C48CE
:106E80006388A7005E24858B81CBA9476316F90030
:106E9000A2852685B5240DEDF24062444A85D24490
:106EA0004249B2490561828097170000938747489D
:106EB0006314F400804469B7971700009387474331
:106EC000E310F4F8C044ADBFA2852685212041D14E
:106ED0007D59D9B741119387418126C2844322C489
:106EE0004AC006C62A892E8489C49C4C99E326850B
:106EF0003526971700009387A741631BF402C04013
:106F00000317C40093170701C18393F68700ADEA06
:106F100093F6070195EEA5472320F90013670704B0
:106F20005AA47D55B24022449244024941018280D4
:106F3000971700009387C73F6314F4008044C9B7D4
:106F4000971700009387C73AE31CF4FAC0444DBF7B
:106F5000918B9DC34C5889C9930744046384F50001
:106F60004A85292B232A04025E242322040093F756
:106F7000B7FD5EA41C481CC05E2493E787005EA496
:106F80001C4899EB5E241307002093F707286385BC
:106F9000E700A2854A8591295E2413F717001DC3D7
:106FA0005C4823240400B307F0401CCC1C48014576
:106FB000B5FB8317C40013F707082DD793E7070421
:106FC0005EA485B7898B014791E3584818C4F9BF7F
:106FD000DE25011122CC26CA06CE4AC84EC613F7BA
:106FE0008700AA842E8479EBD841634DE000B84134
:106FF000634AE0000145F2406244D2444249B2494A
:107000000561828058547DD703A904009396370107
:1070100023A0040063DB060670485E24918B99C7A9
:107020005C401D8E5C5899C33C401D8E5C540C50D6
:10703000814626858297FD575A24631DF5009440AA
:10704000F54763E8D706B70740208507B3D7D700D1
:10705000858BA5C31C48232204001CC0931737014D
:1070600063D80700FD576314F5009C4091E368C89E
:107070004C5823A02401BDDD930744046384F5002C
:107080002685ED2E232A0402B5B70C50014685460D
:1070900026850297FD572A86E311F5F89C40B5DF57
:1070A00075476385E70059476393E70423A02401EC
:1070B00091B7136707045AA47D5535BF83A905010D
:1070C000E38A09F203A905008D8B23A0350133095A
:1070D0003941014791E3D84918C4E35D20F11C54BC
:1070E0000C50CA864E86268582976347A0005E2490
:1070F00093E707045EA4C9B7AA993309A940F1BF71
:107100009C49A5C3011122CC06CE2A8411C51C4D71
:1071100081E72EC62122B245971700009387471FAB
:10712000639CF5004C408397C5009DC7228562444F
:10713000F24005616FF0DFE9971700009387471F62
:107140006394F5000C44C5B7971700009387471A5E
:10715000E39BF5FC4C44C1BFF2406244014505612C
:10716000828001458280411122C406C62A844EA530
:1071700072A52320050023220500232405002322D5
:10718000050623280500232A0500232C0500214697
:1071900081451305C505EF900FBB97170000938736
:1071A00007B35CD097170000938727B51CD49717B7
:1071B0000000938707B95CD497170000938767BBDB
:1071C00000D01CD8B24022444101828097050000C3
:1071D000938545F391AA411126C213068006938434
:1071E000F5FFB384C4024AC02E8922C406C6938523
:1071F00044070D2E2A8401CD2320050023222501DA
:10720000310508C4138684068145EF90CFB32285EB
:10721000B240224492440249410182801C4DA5E7BC
:10722000411106C622C497070000938767FA1CD550
:107230009387C1819C432324050423260504232826
:1072400005046314F50085471CCD2A84352848C001
:1072500022851D2808C42285052848C448400146C7
:107260009145EFF05FF008440546A545EFF0BFEF0C
:1072700048440946C945EFF01FEF85471CCCB24092
:10728000224441018280828041119387C18126C2BC
:1072900084434AC006C69C4C22C42A8981E72685BD
:1072A000EFF0DFF7938484048044DC40FD1763D65D
:1072B00007009C40B9CF8440C5BF0317C40039E71D
:1072C000C17785072322040623200400232204001B
:1072D000232404005CC423280400232A0400232C54
:1072E0000400214681451305C405EF90CFA5232A4C
:1072F0000402232C040223240404232604042285EC
:10730000B24022449244024941018280130484061F
:1073100071BF91454A85EFF01FEC88C049FDB14728
:107320002320F9000144E1BF797122D44AD052CC24
:1073300056CA5AC85EC606D626D24ECE2A8AAE8A0B
:10734000130485040149054BFD5B09ECB25022543E
:107350004A8592540259F249624AD24A424BB24B90
:1073600045618280044483294400FD1963D40900E7
:107370000040E1BFDE24637BFB008397E40063876A
:107380007701A6855285829A3369A9009384840681
:10739000E9BF1971A6DAAE848395E500A2DC86DE2A
:1073A000328463DB0500DE2423A0060093F7070880
:1073B00085E7930700401DA0300836C6EF00F02196
:1073C000B246E34205FE7247BD67F98F7977BA97F7
:1073D00093B717009CC2F1BF930700041CC0F6507E
:1073E0006654D654014509618280DE25011122CC04
:1073F00006CE26CA4AC8898B2E8489CF9307740487
:107400001CC01CC885475CC8F2406244D244424953
:107410000561828074003000AA84EFF09FF7A245D6
:107420002A892685012219E98317C40013F707204A
:1074300061FFF19B93E727005EA4C9B7970700009F
:10744000938707D99CD45E2408C008C893E707082F
:107450005EA4A2475CC8B24781CF8315E4002685AD
:10746000EF00D01A11C55E24F19B93E717005EA4CC
:107470005E243369F9002316240179B7DDC183A79F
:10748000C5FF411122C406C626C21384C5FF63D3BB
:1074900007003E94AA84EF00301F938701989C4315
:1074A00081EF2322040023A081982244B240268544
:1074B000924441016F00701D637EF4001440330755
:1074C000D4006396E7009843DC43369718C05CC04D
:1074D000D9BFBA87D84319C3E37DE4FE944333860A
:1074E000D700631F86001040B29694C33386D7003E
:1074F000E31DC7FA10435843B29694C3D8C375B777
:107500006375C400B1479CC04DB71040B306C400BA
:107510006316D70014435843B29614C058C0C0C372
:1075200069B78280011126CA93843500F19806CE8E
:1075300022CC4AC84EC6A104B14763F3F404B14457
:1075400063E2B4042A89EF003014938701989843CA
:107550003A8439E0938741989C4391E781454A8575
:10756000252F23A2A198A6854A853D27FD59631999
:107570003507B1472320F9004A85EF00101129A0F3
:10758000E3D004FCB1471CC10145F2406244D2443F
:107590004249B249056182801C40858F63CF070252
:1075A000AD4663F6F6001CC03E9404C031A05C40BA
:1075B0006313870223A0F1984A85EF00100D13058D
:1075C000B4009307440061993307F5405DDF3A94B6
:1075D000898F1CC05DBF5CC3C5B72287404095BF83
:1075E000130435007198E30285FCB305A4404A8575
:1075F0006525E31C35FBB5BF1C46FD171CC663DAC9
:107600000700184E63C5E700A9476394F5006FF0C3
:10761000BF801C422E851387170018C28CA382805E
:10762000011122CC26CA4AC84EC652C406CE2A89A7
:10763000AE893284B304D6007D5A631494000145A8
:1076400009A80C204E864A85EFF01FFB0504E316BF
:1076500045FFF2406244D2444249B249224A0561A0
:107660008280357122CD26CB4AC94EC706CF52C57E
:1076700056C35AC1DEDEE2DCE6DAAA89AE8432897C
:10768000368409C51C4D99E3EFF05FB997170000E8
:10769000938707C86398F40C83A44900DE24A18B68
:1076A000E5C79C48F5C393070002A304F1029307C2
:1076B000000302D22305F10222C6930B5002971A4F
:1076C0000000938AEAC8054C294B4A841C2099C3C0
:1076D000639F770DB30C2441638E0C00E6864A86C7
:1076E000A6854E85EFF0DFF3FD57630FF51C92562C
:1076F000E69636D21C206389071CFD571309140037
:1077000002C802CE3ECA02CCA309010482D483453A
:10771000090015465685A92F13041900C24751E9DF
:1077200013F7070109C713070002A309E10413F7C0
:10773000870009C71307B002A309E10483460900C3
:107740001307A002638FE606F2474A848146254666
:10775000182093051400130707FD6377E60AB5CADE
:107760003ECE85A897170000938787BC6395F400E9
:1077700083A4890025B797170000938767B7E39F15
:10778000F4F083A4C90019BFA6854E85EFF08FF4ED
:1077900019D97D55FA406A44DA444A49BA492A4A15
:1077A0009A4A0A4BF65B665CD65C0D6182800504E2
:1077B00031BF330555413315AC00C98F3EC822890E
:1077C000B9B7324793064700184336C663470702E6
:1077D0003ACE18209307E002631DF7041830930790
:1077E000A002631BF702B2470904138747009C43BA
:1077F0003AC663C107023ECA2DA83307E04093E7AB
:1078000027003ACE3EC8F1B7B387670385462E847A
:10781000BA973DBFFD57C5B7050402CA81468147E7
:107820002546182093051400130707FD6374E60628
:10783000F9F20C200D46171500001305E5B10D2DCA
:1078400011CD97170000938727B11D8D9307000472
:10785000B397A700424505045D8D2AC80C20194640
:1078600017150000130585AF130914002304B10296
:10787000012535C19787FFFF9387C77895E7424772
:10788000B2471377071009CF91073EC69257D29798
:107890003ED225BDB387670385462E84BA9751B77C
:1078A0009D07E19BA107D5B7780097060000938656
:1078B00066D726860C084E8597000000E70000007A
:1078C000FD572A8AE314F5FCDE2493F70704E392BC
:1078D00007EC1255C1B5780097060000938686D450
:1078E00026860C084E85012AE1BF797156CA9C494B
:1078F000BA8A984522D426D24ECE52CC06D64AD049
:107900005AC85EC6AA892E84B284368A63D3E70039
:10791000BA879CC00347340419C385079CC01C4028
:1079200093F7070281C79C4089079CC00329040084
:1079300013796900631A0900130B9401FD5B5C4421
:107940009840998F634CF9041C408346340493F7A4
:107950000702B336D000A5EB13063404D2854E855A
:10796000829AFD576303F5041C4011469840998B99
:10797000544481446397C700B384E64063D3040052
:1079800081441C4418486354F700998FBE94014900
:1079900069047D5B63982405014509A885465A86DC
:1079A000D2854E85829A631E75017D55B250225450
:1079B00092540259F249624AD24A424BB24B456153
:1079C00082800509ADBF3307D40013060003A3016D
:1079D000C7040347540493871600A2978906A3811E
:1079E000E7049DBF85462286D2854E85829AE30EA6
:1079F00065FB050945B7797122D426D24AD04ECE0F
:107A000006D652CC56CA5AC8B689942D930790060A
:107A10003289AA842E8413863504638DF60263E2CC
:107A2000D706930780056386F61863EDD700638E4B
:107A3000062093073004638EF60A930A2404230178
:107A4000D404C9A0930730066385F60A930740065D
:107A5000E395F6FE1C40084393F60708930545009E
:107A6000C5C61C410CC363D807001307D002B30777
:107A7000F040A301E404971600009386A68E2947E0
:107A800065A8930700076382F61663E5D70293079C
:107A9000E0066389F6189307F006E390F6FA0C40C7
:107AA0001C4313F80508138547006307080608C33D
:107AB0009C4385A893075007E383F6FE930780074E
:107AC0006389F61293073007E399F6F61C43D04119
:107AD00081459386470014C383AA07005685492E23
:107AE00001C53305554148C05C401CC8A3010404CE
:107AF00061A81C43930A2404938647009C4314C343
:107B00002301F4048547D5B793F607041C410CC341
:107B1000B9DAC207C18781BF93F5050408C3C9D983
:107B20009E231307F0066387E60E971600009386E0
:107B300066832947A30104044C400CC463C50500B7
:107B400008406D9908C099E3B28A89CDB28AB3F52D
:107B5000E702FD1AB6958C212380BA00B3D5E7025F
:107B600063F0E70CA147631EF7001C40858B91CBA7
:107B700058401C4863C7E70093070003A38FFAFE31
:107B8000FD1A3306564110C84E87CA867000A2857A
:107B90002685EFF09FD57D5A631D450B7D55B2506C
:107BA000225492540259F249624AD24A424B4561E8
:107BB0008280A382D504970600009386A67A0C40A3
:107BC000084313F805081C411105630D080208C39A
:107BD00013F7150001C793E505020CC04147B9FB37
:107BE0000C4093F5F5FD0CC0B1B79C4193E707023B
:107BF0009CC193078007A302F404970600009386B4
:107C0000A67775BF13F8050408C3E30308FCC20791
:107C1000C1837DBF970600009386C674214719BFB4
:107C2000AE8735B794411C43CC4913F80608138539
:107C300047006306080008C39C438CC339A008C3EF
:107C400093F606049C43F5DA8EA323280400B28A37
:107C500025BF14485686CA8526858299E30045F5D6
:107C60001C40898B8DE7B2474844E35AF5F23E85C4
:107C70003DB785465686CA8526858299E30065F319
:107C8000050A5C443247998FE345FAFEE9BF014A91
:107C9000930A94017D5BF5B7411122C42A842E8595
:107CA0009707002023A2078806C6EFB0BF92FD57B2
:107CB0006319F50097070020938707879C4391C3BA
:107CC0001CC0B240224441018280411122C42E8452
:107CD0008395E50006C65D2A634905007C48AA979E
:107CE0007CC8B2402244410182805E247D777D17AA
:107CF000F98F5EA4FDB7DE25011122CC26CA4AC841
:107D00004EC606CE93F70710AA842E843289B68910
:107D100091C78395E500894601460D225E247D7753
:107D20007D17F98F5EA48315E4006244F240CE868D
:107D30004A86B24942492685D244056125A84111A7
:107D400022C42E848395E50006C6CD28FD575A240B
:107D5000631AF500FD77FD17F98F5EA4B240224447
:107D6000410182808567D98F5EA468C8C5BF8395AD
:107D7000E50025A8411122C42A842E85B2853686C5
:107D800097F7FF1F23A2077A06C6EFB0DF80FD57E3
:107D90006319F50097F7FF1F938707799C4391C3F9
:107DA0001CC0B240224441018280411122C42A8475
:107DB0002E8597F7FF1F23A9077606C61122FD57C8
:107DC0006319F50097F7FF1F938707769C4391C3CC
:107DD0001CC0B240224441018280411122C42A8445
:107DE0002E85B28597F7FF1F23A0077406C6CD2006
:107DF000FD576319F50097F7FF1F9387E7729C43C0
:107E000091C31CC0B240224441018280411122C46E
:107E10002A842E8597F7FF1F23A8077006C6C9205E
:107E2000FD576319F50097F7FF1F9387E76F9C4392
:107E300091C31CC0B240224441018280411122C43E
:107E40002A842E85B285368697F7FF1F23AE076CEE
:107E500006C67928FD576319F50097F7FF1F93872A
:107E6000A76C9C4391C31CC0B24022444101828054
:107E700093F5F50F2A966314C500014582801C21F5
:107E8000E38EB7FE0505C5BF82808280411122C402
:107E90002A842E85B285368697F7FF1F23A60768AA
:107EA00006C6B928FD576319F50097F7FF1F93879A
:107EB000A7679C4391C31CC0B24022444101828009
:107EC0009307800517F7FF1F2320F7667D558280F3
:107ED0009307800517F7FF1F2328F7647D558280DD
:107EE0009307800517F7FF1F2320F7640145828061
:107EF0009307800517F7FF1F2328F7627D558280BF
:107F00009307800517F7FF1F2320F7627D558280B6
:107F10006D6570633A253038780A00006D636175CD
:107F200073653A253038780A000000006D74766178
:107F30006C3A253038780A0053797374656D436C58
:107F40006B3A25640D0A00004368697049443A257C
:107F50003038780D0A0000005631302E342E3600AD
:107F60004672656552544F53204B65726E656C20A6
:107F700056657273696F6E3A25730D0A0000000032
:107F800073686F756C646E27742072756E206174EF
:107F900020686572652121002E2E2F46726565527C
:107FA000544F532F706F727461626C652F4D656D05
:107FB0004D616E672F686561705F342E630000004D
:107FC000657272206174206C696E65202564206F73
:107FD000662066696C6520222573222E200D0A20FA
:107FE000000000002E2E2F4672656552544F532F0D
:107FF000706F727461626C652F4743432F5249530F
:10800000432D562F706F72742E6300002E2E2F4654
:1080100072656552544F532F71756575652E6300F7
:108020002E2E2F4672656552544F532F7461736B19
:10803000732E630049444C4500000000E03200000C
:10804000E0320000203300002C33000070330000C9
:10805000E0320000E0320000203300002C3300004A
:10806000546D7251000000002E2E2F46726565522D
:10807000544F532F74696D6572732E6300000000B6
:10808000546D7220537663006740533A473C113C6D
:108090006740D33A4A3154696D6572004A32546977
:1080A0006D6572004A3354696D6572004A345469D3
:1080B0006D6572004A355F3054696D65720000006D
:1080C0005B494E464F5D205B25733A25645D207801
:1080D000506F727447657446726565486561705388
:1080E000697A65203A2025640D0A0000636F6D6D82
:1080F0006F6E5461736B00007472616E736D69749E
:108100005461736B000000005570526563656976B9
:10811000655461736B000000446F776E5265636550
:108120006976655461736B00467265654D656D6F68
:1081300072795461736B0000000020415B494E4628
:108140004F5D205B25733A25645D20696E2047579B
:108150005F4D736750726F6346756E635F446973FA
:10816000747269627574696F6E5F50726F66696C64
:10817000650A0D0A000000005B494E464F5D205B1A
:1081800025733A25645D20696E2047575F4D7367FC
:1081900050726F6346756E635F526561645F5072C3
:1081A0006F66696C650A0D0A00000000C2E7FFFFF8
:1081B00014E7FFFF14E7FFFF12E7FFFF18E7FFFFD9
:1081C00018E7FFFFE8E6FFFF12E7FFFF18E7FFFFF2
:1081D000E8E6FFFF18E7FFFF12E7FFFFB0E7FFFF4A
:1081E000B0E7FFFFB0E7FFFFE8E6FFFF0001020294
:1081F000030303030404040404040404050505053F
:10820000050505050505050505050505060606061A
:1082100006060606060606060606060606060606FE
:1082200006060606060606060606060607070707EA
:1082300007070707070707070707070707070707CE
:1082400007070707070707070707070707070707BE
:1082500007070707070707070707070707070707AE
:10826000070707070707070707070707080808089A
:10827000080808080808080808080808080808087E
:10828000080808080808080808080808080808086E
:10829000080808080808080808080808080808085E
:1082A000080808080808080808080808080808084E
:1082B000080808080808080808080808080808083E
:1082C000080808080808080808080808080808082E
:1082D000080808080808080808080808080808081E
:1082E000080808080808080808080808000000002E
:1082F000000000000000000000000000000000007E
:10830000000000000000000000000000000000006D
:10831000000000000000000000000000000000005D
:10832000000000000000000000000000000000004D
:10833000000000000000000000000000000000003D
:10834000000000000000000000000000232D302B82
:1083500020000000686C4C006566674546470000D9
:10836000303132333435363738394142434445466B
:10837000000000003031323334353637383961622D
:08838000636465660000000063
:1083880000000000000000000102030406070809BD
:1083980000000000010203040102030406070809A3
:1083A800000000000600000080250000000000001A
:1083B80000000000000000000000000000000000B5
:1083C80000000000000000000700000080250000F9
:1083D8000000000000000000000000000000000095
:1083E8000000000000000000000000000200000083
:1083F80080250000000000000000000000000000D0
:108408000000000000000000000000000000000064
:1084180008000000802500000000000000000000A7
:108428000000000000000000000000000000000044
:10843800000000000300000080250000000000008C
:108448000000000000000000000000000000000024
:1084580000000000000000000500000000C201004C
:108468000000000000000000000000000000000004
:108478000000000000000000000000001C5F000079
:1084880001000000FC5E000002000000DC5E00004D
:1084980003000000CE5E000004000000C05E000083
:1084A80005000000B25E000006000000A45E0000A7
:1084B80007000000965E000008000000885E0000CB
:1084C800090000007A5E00000A0000006C5E0000EF
:1084D8000B0000005E5E000003000000CC5F00009F
:1084E80004000000BA5F000005000000A85F00005B
:1084F80006000000965F000007000000845F00008F
:1085080008000000725F000009000000605F0000C2
:108518000A0000004E5F00000B0000003C5F0000F6
:10852800000000000C8300002C830000EC82000097
:108538000000000000000000000000000000000033
:108548000000000000000000000000000000000023
:108558000000000000000000000000000000000013
:108568000000000000000000000000000000000003
:1085780000000000000000000000000000000000F3
:10858800006CDC0202040608AAAAAAAA09000000D4
:1085980028750020A001002000800020A0010020F4
:00000001FF
